:020000040000FA
:1000000000020400000000003C6E0000486E00008A
:10001000546E0000606E00006C6E0000786E000090
:10002000846E00009C6E0000906E0000906E0000D8
:10003000906E0000906E0000906E0000906E0000C8
:10004000906E00000C700000906E0000906E00003A
:10005000906E0000366A0000906E0000906E000006
:10006000906E0000906E0000906E0000906E000098
:10007000906E0000906E0000906E0000906E000088
:10008000906E0000906E0000906E0000906E000078
:10009000906E0000906E0000906E0000906E000068
:1000A000906E0000F06C0000906E0000906E0000FA
:1000B000906E0000906E0000906E0000906E000048
:1000C000906E0000906E0000906E0000906E000038
:1000D000906E0000906E0000906E0000906E000028
:1000E000906E0000906E0000906E0000906E000018
:1000F000906E0000906E0000906E0000906E000008
:10010000906E0000906E0000906E0000906E0000F7
:10011000906E0000906E0000906E0000906E0000E7
:10012000906E0000906E0000906E0000066D000062
:100130000C6D0000906E0000906E0000906E00004C
:10014000906E0000906E0000906E0000906E0000B7
:10015000906E0000906E0000906E0000906E0000A7
:10016000906E0000906E0000906E00003E6D0000EA
:10017000126D0000286D0000906E0000906E00006F
:10018000906E0000906E0000906E0000906E000077
:10019000906E0000906E0000906E0000906E000067
:1001A000906E0000906E0000906E0000906E000057
:1001B000906E0000906E0000906E0000906E000047
:1001C000906E0000906E0000906E0000906E000037
:1001D000906E0000906E0000906E0000906E000027
:1001E000906E0000906E0000906E0000906E000017
:1001F000906E0000906E0000906E0000906E000007
:10020000906E0000906E0000906E0000906E0000F6
:10021000906E0000906E0000906E0000906E0000E6
:10022000906E0000906E0000906E0000906E0000D6
:10023000906E0000906E0000906E0000906E0000C6
:10024000906E0000906E0000906E0000906E0000B6
:10025000906E0000906E0000906E0000906E0000A6
:10026000906E0000906E0000FFFFFF00FFFFFF0098
:10027000FFFFFF00FFFFFF00FFFFFF00FFFFFF008A
:10028000FFFFFF00FFFFFF00FFFFFF00FFFFFF007A
:10029000FFFFFF00FFFFFF00FFFFFF00FFFFFF006A
:1002A000FFFFFF00FFFFFF00FFFFFF00FFFFFF005A
:1002B000FFFFFF00FFFFFF00FFFFFF00FFFFFF004A
:1002C000FFFFFF00FFFFFF00FFFFFF00FFFFFF003A
:1002D000FFFFFF00FFFFFF00FFFFFF00FFFFFF002A
:1002E000FFFFFF00FFFFFF00FFFFFF00FFFFFF001A
:1002F000FFFFFF00FFFFFF00FFFFFF00FFFFFF000A
:10030000FFFFFF00FFFFFF00FFFFFF00FFFFFF00F9
:10031000FFFFFF00FFFFFF00FFFFFF00FFFFFF00E9
:10032000FFFFFF00FFFFFF00FFFFFF00FFFFFF00D9
:10033000FFFFFF00FFFFFF00FFFFFF00FFFFFF00C9
:10034000FFFFFF00FFFFFF00FFFFFF00FFFFFF00B9
:10035000FFFFFF00FFFFFF00FFFFFF00FFFFFF00A9
:10036000FFFFFF00FFFFFF00FFFFFF00FFFFFF0099
:10037000FFFFFF00FFFFFF00FFFFFF00FFFFFF0089
:10038000FFFFFF00FFFFFF00FFFFFF00FFFFFF0079
:10039000FFFFFF00FFFFFF00FFFFFF00FFFFFF0069
:1003A000FFFFFF00FFFFFF00FFFFFF00FFFFFF0059
:1003B000FFFFFF00FFFFFF00FFFFFF00FFFFFF0049
:1003C000FFFFFF00FFFFFF00FFFFFF00FFFFFF0039
:1003D000FFFFFF00FFFFFF00FFFFFF00FFFFFF0029
:1003E000FFFFFF00FFFFFF00FFFFFF00FFFFFF0019
:1003F000FFFFFF00FFFFFF00FFFFFF00FFFFFF0009
:100400004FEB210080F12100000188000000000076
:1004100038620200000000000000200040708800E8
:10042000000020005070880000002000307088001C
:1004300000002000607088000000200070708800BC
:10044000000020000070880000002000207088005C
:1004500000002000C070880000002000D0708800DC
:1004600000002000E070880000002000F07088008C
:10047000F00F20008070880000002000A07088002D
:1004800000002000407188000000200050718800AA
:10049000000020006071880000002000707188005A
:1004A000E0012F000071880000002000207188000A
:1004B00000002000C071880000002000D07188007A
:1004C00000032300B071880000002000E071880064
:1004D00000002000F0718800000024008071880076
:1004E00080032300A0718800000020004072880073
:1004F0000000200050728800000020006072880018
:100500000000200070728800200020000072880027
:10051000100820002072880000002000C0728800AF
:1005200000002000D072880000002300B072880014
:1005300000002000E0728800000222008072880023
:1005400000012100A0728800000020004073880094
:1005500000002000507388003000240030738800B1
:100560000000200060738800000020007073880085
:1005700020082000007388001000200020738800ED
:1005800000002000C0738800F0CF2000D0738800E6
:1005900000002000B073880000002000E073880095
:1005A000F0CF20008073880000002000A073880036
:1005B000000020004074880000002700507488006C
:1005C000F00F200030748800000020006074880064
:1005D00000002700007488000000280020748800B4
:1005E00000002000C074880000002000D074880043
:1005F00000002000B074880000002000E074880033
:10060000000022008074880000002C00A074880084
:1006100010032000203688001005200030368800A6
:10062000D0062000B036880010072000C0368800B1
:100630000030200040348800001020006034880022
:1006400000B02100B034880000D02100C034880000
:1006500010302300103A880020002000203A880043
:10066000A0082000303A880075AEA80075CEA8001A
:1006700000802A0000118800004C22001011880020
:10068000701C20004011880000802A008011880022
:10069000004C22009011880060022000C0118800E8
:1006A00060802A008012880000402000901288009C
:1006B000701C2000C012880060802A00801588000D
:1006C000004C200090158800701C2000C015880088
:1006D000158EA80004CEA90080072100A083880001
:1006E000B0838800401A2100008D8800108D88009A
:1006F0008020210020908800309088000014210084
:10070000E0898800F0898800C08D2100C0C688007B
:10071000D0C68800000228008008880050442000CD
:1007200060088800C838EF00CE38EF00F0FF2F00D7
:1007300080C6880090C688000230EF006988A90052
:1007400069A8A90069C8A8006888A80068A8A900C5
:1007500068C8A8004388A80043A8A90043C8A80007
:10076000646102000000000065CEA8006461020020
:100770000000000000042000C6620200000000002B
:100780000003200044620200000000007008200006
:100790004462020000000000700020004462020079
:1007A000000000007002200044620200000000000F
:1007B000F00220004462020000000000F00E200061
:1007C0004462020000000000800220004462020037
:1007D0000000000000002000446202000000000051
:1007E00040042000C662020000000000000020005B
:1007F0004462020000000000000020004462020089
:1008000000000000000F2000446202000000000011
:100810000008200044620200000000005002200096
:100820004462020000000000000F20004462020049
:1008300000000000000020004462020000000000F0
:10084000B00420004462020000000000000020000C
:100850004462020000000000000020004462020028
:1008600000000000A0052000C66202000000000099
:10087000000020004462020000000000B0052000DB
:10088000C662020000000000100020004462020066
:100890000000000080052000C66202000000000089
:1008A0006005200044620200000000009E63020018
:1008B0000000000060042000C6620200000000008A
:1008C0000000200044620200000000000000200040
:1008D0004462020000000000D0052000C662020051
:1008E0000000000040002000446202000000000000
:1008F000700020004462020000000000900520000B
:10090000C662020000000000C0042000C6620200AF
:1009100000000000154EA80015EEA90015CEA90094
:1009200015AEA8000000000000000000000000005C
:1009300000000000000000000000000000000000B7
:10094000152EA800CC61020000000000CC6102005E
:1009500000000000CC61020000000000CC61020039
:10096000000000000A61020000000000CC610200EB
:1009700000000000CC61020000000000CC61020019
:1009800000000000CC6102000000000015EEA8008D
:1009900015CEA80015AEA800000000000000000061
:1009A0000000000000000000000000000000000047
:1009B00000000000152EA800CC610200000000001D
:1009C000CC61020000000000CC61020000000000C9
:1009D000CC610200000000000A610200000000007B
:1009E000CC61020000000000CC61020000000000A9
:1009F000CC61020000000000CC6102000000000099
:100A000015EEA90015CEA90015AEA9000000000042
:100A100000000000000000000000000000000000D6
:100A20000000000000000000152EA800CC610200AC
:100A300000000000CC61020000000000CC61020058
:100A400000000000CC610200000000000A6102000A
:100A500000000000CC61020000000000CC61020038
:100A600000000000CC61020000000000CC61020028
:100A700000000000156EA90000000000000000004A
:100A80000000000000000000000000000000000066
:100A900000000000800E20002C600200000000001A
:100AA000000020002C600200000000000000200078
:100AB0002C60020000000000000020002C600200FA
:100AC00000000000000020002C6002000000000078
:100AD000000020002C600200000000000000200048
:100AE0002C60020000000000000020002C600200CA
:100AF000000000008060020000000000000278009A
:100B000080600200000000004800DD00040040009A
:100B1000F080880080600200000000000002780081
:100B200080600200000000004800DD00040040007A
:100B30000081880080600200000000000002780050
:100B400080600200000000004800DD00040040005A
:100B5000008388008060020000000000000278002E
:100B600080600200000000004800DD00040040003A
:100B700010838800806002000000000000027800FE
:100B800080600200000000004800DD00040040001A
:100B900020838800806002000000000000027800CE
:100BA00080600200000000004800DD0004004000FA
:100BB000308388008060020000000000000278009E
:100BC00080600200000000004800DD0004004000DA
:100BD000408388008060020000000000000278006E
:100BE00080600200000000004800DD0004004000BA
:100BF00001052000810050004220AF000E060400D5
:100C00000000000031042000810050004220AF00AD
:100C10000E0604000000000000052000508388003C
:100C20008060020000000000000278008060020086
:100C3000000000004800DD000400400060838800E0
:100C40008060020000000000000278008060020066
:100C5000000000004800DD0004004000E080880043
:100C60008060020000000000000278008060020046
:100C7000000000004800DD0004004000E093880010
:100C80008060020000000000000278008060020026
:100C9000000000004800DD0004004000F0938800E0
:100CA000156EA80000000000000000000000000019
:100CB0000000000000000000000000000000000034
:100CC00015EEA80015CEA80015AEA8000000000083
:100CD0000000000000000000000000000000000014
:100CE0000000000000000000156EA90000000000D8
:100CF00000000000000000000000000000000000F4
:100D00000000000000000000800E20002C600200A7
:100D100000000000000020002C6002000000000025
:100D2000000020002C6002000000000000002000F5
:100D30002C60020000000000000020002C60020077
:100D400000000000000020002C60020000000000F5
:100D5000000020002C6002000000000000002000C5
:100D60002C60020000000000806002000000000013
:100D70000002780080600200000000004800DD00F2
:100D80000400400000948800806002000000000021
:100D90000002780080600200000000004800DD00D2
:100DA0000400400010948800156EA80000000000A8
:100DB0000000000000000000000000000000000033
:100DC0000000000000000000862821001000200024
:100DD000005B780050032000005B780000838000F7
:100DE000001B7800A0002000001B780000002000FD
:100DF000001B7800000A2000001B7800A6292100B3
:100E000000002000001B780000402600001B780036
:100E1000A62B210010002000005B7800500320006A
:100E2000005B780000838000001B7800A000200099
:100E3000001B780000002000001B7800000F20003D
:100E4000001B7800C62C210000002000001B780049
:100E500000402600001B7800C62E21001000200054
:100E6000005B780050032000005B78000083800066
:100E7000001B7800A0002000001B7800000020006C
:100E8000001B780000142000001B7800E62F2100D2
:100E900000002000001B780000402600001B7800A6
:100EA000E631210010002000005B78005003200094
:100EB000005B780000838000001B7800A000200009
:100EC000001B780000002000001B780000192000A3
:100ED000001B78000633210000002000001B780072
:100EE00000402600001B780006352100100020007D
:100EF000005B780050032000005B780000838000D6
:100F0000001B7800A0002000001B780000002000DB
:100F1000001B7800001E2000001B780026362100F0
:100F200000002000001B780000402600001B780015
:100F30002638210010002000005B780050032000BC
:100F4000005B780000838000001B7800A000200078
:100F5000001B780000002000001B78000023200008
:100F6000001B78004639210000002000001B78009B
:100F700000402600001B7800463B210010002000A6
:100F8000005B780050032000005B78000083800045
:100F9000001B7800A0002000001B7800000020004B
:100FA000001B780000282000001B7800663C210010
:100FB00000002000001B780000402600001B780085
:100FC000663E210010002000005B780050032000E6
:100FD000005B780000838000001B7800A0002000E8
:100FE000001B780000002000001B7800002D20006E
:100FF000001B7800863F210000002000001B7800C5
:1010000000402600001B78008641210010002000CF
:10101000005B780050032000005B780000838000B4
:10102000001B7800A0002000001B780000002000BA
:10103000001B7800002D2000001B7800A642210034
:1010400000002000001B780000402600001B7800F4
:10105000A644210010002000005B7800500320000F
:10106000005B780000838000001B7800A000200057
:10107000001B780000002000001B7800002D2000DD
:10108000001B7800C645210000002000001B7800EE
:1010900000402600001B7800C647210010002000F9
:1010A000005B780050032000005B78000083800024
:1010B000001B7800A0002000001B7800000020002A
:1010C000001B7800002D2000001B7800E64821005E
:1010D00000002000001B780000402600001B780064
:1010E000E64A210010002000005B78005003200039
:1010F000005B780000838000001B7800A0002000C7
:10110000001B780000002000001B7800002D20004C
:10111000001B7800064C210000002000001B780016
:1011200000402600001B7800064E21001000200021
:10113000005B780050032000005B78000083800093
:10114000001B7800A0002000001B78000000200099
:10115000001B7800002D2000001B7800264F210086
:1011600000002000001B780000402600001B7800D3
:101170002651210010002000005B78005003200061
:10118000005B780000838000001B7800A000200036
:10119000001B780000002000001B7800002D2000BC
:1011A000001B78004652210000002000001B780040
:1011B00000402600001B780046542100100020004B
:1011C000005B780050032000005B78000083800003
:1011D000001B7800A0002000001B78000000200009
:1011E000001B7800002D2000001B780066552100B0
:1011F00000002000001B780000402600001B780043
:101200006657210010002000005B7800500320008A
:10121000005B780000838000001B7800A0002000A5
:10122000001B780000002000001B7800002D20002B
:10123000001B78008658210000002000001B780069
:1012400000402600001B7800865A21001000200074
:10125000005B780050032000005B78000083800072
:10126000001B7800A0002000001B78000000200078
:10127000001B7800002D2000001B7800A65B2100D9
:1012800000002000001B780000402600001B7800B2
:10129000A65D210010002000005B780050032000B4
:1012A000005B780000838000001B7800A000200015
:1012B000001B780000002000001B7800002D20009B
:1012C000001B7800C65E210000002000001B780093
:1012D00000402600001B7800C6602100100020009E
:1012E000005B780050032000005B780000838000E2
:1012F000001B7800A0002000001B780000002000E8
:10130000001B7800002D2000001B7800E661210002
:1013100000002000001B780000402600001B780021
:10132000E663210010002000005B780050032000DD
:10133000005B780000838000001B7800A000200084
:10134000001B780000002000001B7800002D20000A
:10135000001B78000665210000002000001B7800BB
:1013600000402600001B78000667210010002000C6
:10137000005B780050032000005B78000083800051
:10138000001B7800A0002000001B78000000200057
:10139000001B7800002D2000001B7800266821002B
:1013A00000002000001B780000402600001B780091
:1013B000266A210010002000005B78005003200006
:1013C000005B780000838000001B7800A0002000F4
:1013D000001B780000002000001B7800002D20007A
:1013E000001B7800466B210000002000001B7800E5
:1013F00000402600001B7800466D210010002000F0
:10140000005B780050032000005B780000838000C0
:10141000001B7800A0002000001B780000002000C6
:10142000001B7800002D2000001B7800666E210054
:1014300000002000001B780000402600001B780000
:101440006670210010002000005B7800500320002F
:10145000005B780000838000001B7800A000200063
:10146000001B780000002000001B7800002D2000E9
:10147000001B78008671210000002000001B78000E
:1014800000402600001B7800867321001000200019
:10149000005B780050032000005B78000083800030
:1014A000001B7800A0002000001B78000000200036
:1014B000001B7800002D2000001B7800A67421007E
:1014C00000002000001B780000402600001B780070
:1014D000A676210010002000005B78005003200059
:1014E000005B780000838000001B7800A0002000D3
:1014F000001B780000002000001B7800002D200059
:10150000001B7800C677210000002000001B780037
:1015100000402600001B7800C67921001000200042
:10152000005B780050032000005B7800008380009F
:10153000001B7800A0002000001B780000002000A5
:10154000001B7800002D2000001B7800E67A2100A7
:1015500000002000001B780000402600001B7800DF
:10156000E67C210010002000005B78005003200082
:10157000005B780000838000001B7800A000200042
:10158000001B780000002000001B7800002D2000C8
:10159000001B7800067E210000002000001B780060
:1015A00000402600001B780006802100100020006B
:1015B000005B780050032000005B7800008380000F
:1015C000001B7800A0002000001B78000000200015
:1015D000001B7800002D2000001B780026812100D0
:1015E00000002000001B780000402600001B78004F
:1015F0002683210010002000005B780050032000AB
:10160000005B780000838000001B7800A0002000B1
:10161000001B780000002000001B7800002D200037
:10162000001B78004684210000002000001B780089
:1016300000402600001B7800468621001000200094
:10164000005B780050032000005B7800008380007E
:10165000001B7800A0002000001B78000000200084
:10166000001B7800002D2000001B780066872100F9
:1016700000002000001B780000402600001B7800BE
:101680006689210010002000005B780050032000D4
:10169000005B780000838000001B7800A000200021
:1016A000001B780000002000001B7800002D2000A7
:1016B000001B7800868A210000002000001B7800B3
:1016C00000402600001B7800B46702000000000004
:1016D000F00F200040938800803E20008083880027
:1016E0000000200010818800208188000000200078
:1016F000609388002828A8002848A8002A28A80065
:101700002168A8002A48A80020E8A800C228A8004C
:1017100000002000B0C688000230AE00161204009F
:10172000000000000230A900B0072000E66F0200B0
:101730000000000080B02E00E66F020000000000F4
:1017400000838000E66F020000000000108380002C
:10175000E66F02000000000020838000E66F0200B8
:101760000000000030838000E66F020000000000EF
:1017700040838000E66F020000000000508380007C
:10178000E66F02000000000060838000E66F020048
:1017900000000000F0808000E66F02000000000002
:1017A00000818000E66F020000000000E080800001
:1017B000E66F02000000000070838000E66F020008
:1017C00000000000F0828000E66F020000000000D0
:1017D0008628210016027800F10F20000102620025
:1017E00041012000068340009641780001F02F005F
:1017F0008181610004807100E66F0200000000003A
:1018000086282100200220000003430016007800F3
:10181000E66F020000000000A62B210016027800EF
:10182000F10F200001026200410120000683400008
:101830009641780001F02F008181610004807100E1
:10184000E66F020000000000A62B2100200220000D
:101850000003430016007800E66F0200000000005D
:10186000C62E210016027800F10F2000010262004E
:1018700041012000068340009641780001F02F00CE
:101880008181610004807100E66F020000000000A9
:10189000C62E21002002200000034300160078001D
:1018A000E66F020000000000E63121001602780019
:1018B000F10F200001026200410120000683400078
:1018C0009641780001F02F00818161000480710051
:1018D000E66F020000000000E63121002002200037
:1018E0000003430016007800E66F020000000000CD
:1018F0000635210016027800F10F20000102620077
:1019000041012000068340009641780001F02F003D
:101910008181610004807100E66F02000000000018
:101920000635210020022000000343001600780045
:10193000E66F020000000000263821001602780041
:10194000F10F2000010262004101200006834000E7
:101950009641780001F02F008181610004807100C0
:10196000E66F02000000000026382100200220005F
:101970000003430016007800E66F0200000000003C
:10198000463B210016027800F10F200001026200A0
:1019900041012000068340009641780001F02F00AD
:1019A0008181610004807100E66F02000000000088
:1019B000463B21002002200000034300160078006F
:1019C000E66F020000000000663E2100160278006B
:1019D000F10F200001026200410120000683400057
:1019E0009641780001F02F00818161000480710030
:1019F000E66F020000000000663E21002002200089
:101A00000003430016007800E66F020000000000AB
:101A10008641210016027800F10F200001026200C9
:101A200041012000068340009641780001F02F001C
:101A30008181610004807100E66F020000000000F7
:101A40008641210020022000000343001600780098
:101A5000E66F020000000000A64421001602780094
:101A6000F10F2000010262004101200006834000C6
:101A70009641780001F02F0081816100048071009F
:101A8000E66F020000000000A644210020022000B2
:101A90000003430016007800E66F0200000000001B
:101AA000C647210016027800F10F200001026200F3
:101AB00041012000068340009641780001F02F008C
:101AC0008181610004807100E66F02000000000067
:101AD000C6472100200220000003430016007800C2
:101AE000E66F020000000000E64A210016027800BE
:101AF000F10F200001026200410120000683400036
:101B00009641780001F02F0081816100048071000E
:101B1000E66F020000000000E64A210020022000DB
:101B20000003430016007800E66F0200000000008A
:101B3000064E210016027800F10F2000010262001B
:101B400041012000068340009641780001F02F00FB
:101B50008181610004807100E66F020000000000D6
:101B6000064E2100200220000003430016007800EA
:101B7000E66F0200000000002651210016027800E6
:101B8000F10F2000010262004101200006834000A5
:101B90009641780001F02F0081816100048071007E
:101BA000E66F020000000000265121002002200004
:101BB0000003430016007800E66F020000000000FA
:101BC0004654210016027800F10F20000102620045
:101BD00041012000068340009641780001F02F006B
:101BE0008181610004807100E66F02000000000046
:101BF0004654210020022000000343001600780014
:101C0000E66F02000000000066572100160278000F
:101C1000F10F200001026200410120000683400014
:101C20009641780001F02F008181610004807100ED
:101C3000E66F02000000000066572100200220002D
:101C40000003430016007800E66F02000000000069
:101C5000865A210016027800F10F2000010262006E
:101C600041012000068340009641780001F02F00DA
:101C70008181610004807100E66F020000000000B5
:101C8000865A21002002200000034300160078003D
:101C9000E66F020000000000A65D21001602780039
:101CA000F10F200001026200410120000683400084
:101CB0009641780001F02F0081816100048071005D
:101CC000E66F020000000000A65D21002002200057
:101CD0000003430016007800E66F020000000000D9
:101CE000C660210016027800F10F20000102620098
:101CF00041012000068340009641780001F02F004A
:101D00008181610004807100E66F02000000000024
:101D1000C660210020022000000343001600780066
:101D2000E66F020000000000E66321001602780062
:101D3000F10F2000010262004101200006834000F3
:101D40009641780001F02F008181610004807100CC
:101D5000E66F020000000000E66321002002200080
:101D60000003430016007800E66F02000000000048
:101D70000667210016027800F10F200001026200C0
:101D800041012000068340009641780001F02F00B9
:101D90008181610004807100E66F02000000000094
:101DA000066721002002200000034300160078008F
:101DB000E66F020000000000266A2100160278008B
:101DC000F10F200001026200410120000683400063
:101DD0009641780001F02F0081816100048071003C
:101DE000E66F020000000000266A210020022000A9
:101DF0000003430016007800E66F020000000000B8
:101E0000466D210016027800F10F200001026200E9
:101E100041012000068340009641780001F02F0028
:101E20008181610004807100E66F02000000000003
:101E3000466D2100200220000003430016007800B8
:101E4000E66F0200000000006670210016027800B4
:101E5000F10F2000010262004101200006834000D2
:101E60009641780001F02F008181610004807100AB
:101E7000E66F0200000000006670210020022000D2
:101E80000003430016007800E66F02000000000027
:101E90008673210016027800F10F20000102620013
:101EA00041012000068340009641780001F02F0098
:101EB0008181610004807100E66F02000000000073
:101EC00086732100200220000003430016007800E2
:101ED000E66F020000000000A676210016027800DE
:101EE000F10F200001026200410120000683400042
:101EF0009641780001F02F0081816100048071001B
:101F0000E66F020000000000A676210020022000FB
:101F10000003430016007800E66F02000000000096
:101F2000C679210016027800F10F2000010262003C
:101F300041012000068340009641780001F02F0007
:101F40008181610004807100E66F020000000000E2
:101F5000C67921002002200000034300160078000B
:101F6000E66F020000000000E67C21001602780007
:101F7000F10F2000010262004101200006834000B1
:101F80009641780001F02F0081816100048071008A
:101F9000E66F020000000000E67C21002002200025
:101FA0000003430016007800E66F02000000000006
:101FB0000680210016027800F10F20000102620065
:101FC00041012000068340009641780001F02F0077
:101FD0008181610004807100E66F02000000000052
:101FE0000680210020022000000343001600780034
:101FF000E66F020000000000268321001602780030
:10200000F10F200001026200410120000683400020
:102010009641780001F02F008181610004807100F9
:10202000E66F02000000000026832100200220004D
:102030000003430016007800E66F02000000000075
:102040004686210016027800F10F2000010262008E
:1020500041012000068340009641780001F02F00E6
:102060008181610004807100E66F020000000000C1
:10207000468621002002200000034300160078005D
:10208000E66F020000000000668921001602780059
:10209000F10F200001026200410120000683400090
:1020A0009641780001F02F00818161000480710069
:1020B000E66F020000000000668921002002200077
:1020C0000003430016007800E66F020000000000E5
:1020D00020808000E66F0200000000003080800059
:1020E000E66F02000000000040808000E66F020002
:1020F0000000000050808000E66F02000000000039
:1021000060808000E66F02000000000070808000A8
:10211000E66F02000000000080808000E66F020091
:102120000000000090808000E66F020000000000C8
:10213000A0808000E66F020000000000B0808000F8
:10214000E66F020000000000C0808000E66F020021
:1021500000000000D0808000E66F02000000000058
:10216000D0072000E66F02000000000000402000C1
:10217000B1C68000808050004200AE0016120400FC
:1021800000000000E093800020948800F09380001D
:102190003094880000948000E093880010948000C0
:1021A000F093880015EEA90015CEA90015AEA80081
:1021B000000000000000000000000000000000001F
:1021C0000000000000000000000000007077020026
:1021D00000000000156EA9000000000000000000D3
:1021E00000000000000000000000000000000000EF
:1021F00000000000400820002C60020000000000E9
:10220000F4938000F3072000030062002C600200BA
:1022100000000000E49380004822DE00030062001A
:102220002C60020000000000E4938000F30F200007
:10223000030062002C600200000000000620200065
:10224000FA6F020000000000000278004800DE0083
:10225000F30F2000030060002C600200000000006B
:10226000030062002C600200000000000603E90089
:102270000600E0004220AE00201104000000000033
:10228000000000000000000000000000156EA80023
:10229000000000000000000000000000000000003E
:1022A000000000000000000000000000CC610200FF
:1022B00000000000CC770200000000000040200079
:1022C00001002000E2938000F393800002004000B0
:1022D000838048000094880011948800000020004A
:1022E000E093880000002000F093880015EEA8001D
:1022F00015CEA80015AEA8000000000000000000E8
:1023000000000000000000000000000000000000CD
:10231000000000007077020000000000156EA900A8
:1023200000000000000000000000000000000000AD
:102330000000000000000000000000004008200035
:102340002C60020000000000000020002C60020051
:1023500000000000000020002C60020000000000CF
:10236000000020002C6002000000000000948000AB
:1023700000027800F30F2000030060002C600200D0
:10238000000000004822DE00030062002C60020012
:10239000000000001094800000027800F30F20007D
:1023A000030060002C600200000000004822DE00F4
:1023B000030062002C60020000000000156EA800FF
:1023C000000000000000000000000000000000000D
:1023D000000000000000000000000000CC610200CE
:1023E00000000000CC7702000000000015EEA900FC
:1023F00015CEA90015AEA9000000000000000000E5
:1024000000000000000000000000000000000000CC
:102410000000000020948000E09388003094800049
:10242000F093880000402000D638B500108180006D
:102430000000D000E107200001006000000601005C
:1024400066140400000000001417040000000000DF
:102450001E17040000000000161B0400000000000E
:102460009A480400000000001E4B04000000000019
:10247000A4130400000000004A140400000000003F
:102480007E2104000000000014270400000000006A
:10249000484D0400000000008054040000000000CB
:1024A000F44004000000000010440400000000009C
:1024B000C427040000000000E02804000000000021
:1024C000B42E040000000000D4340400000000001A
:1024D000142A040000000000302B0400000000005B
:1024E000642C040000000000802D040000000000A7
:1024F000783504000000000094360400000000005D
:10250000C837040000000000E438040000000000A8
:10251000183A040000000000343B040000000000F2
:10252000683C040000000000843D0400000000003E
:10253000A43E040000000000C03F040000000000B2
:10254000484404000000000064450400000000004E
:1025500098460400000000005C48040000000000F1
:102560009C130400000000009C1304000000000005
:102570009C130400000000009C13040000000000F5
:102580009C130400000000009C13040000000000E5
:102590009C130400000000009C13040000000000D5
:1025A0009C130400000000009C13040000000000C5
:1025B0009C130400000000009C13040000000000B5
:1025C0009C130400000000009C13040000000000A5
:1025D0009C130400000000009C1304000000000095
:1025E0009C130400000000009C1304000000000085
:1025F0009C130400000000009C1304000000000075
:102600009C130400000000009C1304000000000064
:102610009C130400000000009C1304000000000054
:102620009C130400000000009C1304000000000044
:102630009C130400000000009C1304000000000034
:102640009C130400000000009C1304000000000024
:102650009C130400000000009C1304000000000014
:102660009C130400000000009C1304000000000004
:102670009C130400000000009C13040000000000F4
:102680009C130400000000009C13040000000000E4
:102690009C130400000000009C13040000000000D4
:1026A0009C130400000000009C13040000000000C4
:1026B0009C130400000000009C13040000000000B4
:1026C0009C130400000000009C13040000000000A4
:1026D0009C130400000000009C1304000000000094
:1026E0009C130400000000009C1304000000000084
:1026F0009C130400000000009C1304000000000074
:102700009C130400000000009C1304000000000063
:102710009C130400000000009C1304000000000053
:102720009C130400000000009C1304000000000043
:102730009C130400000000000000200010818800AD
:102740008C0B0400000000009E63020000000000EB
:10275000E411200060042000C662020000000000B6
:10276000F30F20000300620044620200000000003A
:102770004822DE0003006200446202000000000004
:1027800020042000C6620200000000003005200086
:1027900044620200000000000002200044620200C7
:1027A000000000004005200044620200000000001C
:1027B00000022000446202000000000050052000DA
:1027C0004462020000000000000220004462020097
:1027D000000000002004200044620200000000000D
:1027E0008448200060042000C6620200000000004F
:1027F000F30F2000030062004462020000000000AA
:102800004822DE0003006200446202000000000073
:1028100020042000C662020000000000D004200056
:102820004462020000000000100420004462020024
:10283000000000009004200044620200000000003C
:10284000E0042000446202000000000000022000BA
:102850004462020000000000D00420004462020034
:10286000000000005004200044620200000000004C
:10287000E004200044620200000000005005200037
:1028800044620200000000002230EC008C0B0400C7
:102890000000000090C680003100200001005000C0
:1028A0004220AE006214040000000000702102000B
:1028B0000000000020002000108188008C0B040024
:1028C000000000008C0B0400000000009E6302006A
:1028D000000000006417200060042000C6620200AF
:1028E00000000000F30F20000300620044620200B9
:1028F000000000004822DE00030062004462020083
:102900000000000020042000C66202000000000059
:1029100010042000446202000000000000022000B9
:1029200044620200000000007004200044620200C3
:1029300000000000000220004462020000000000CD
:102940002005200044620200000000000002200078
:102950004462020000000000900420004462020073
:10296000000000000002200044620200000000009D
:1029700070042000446202000000000000022000F9
:102980004462020000000000500420004462020083
:10299000000000000002200044620200000000006D
:1029A000C004200044620200000000004421200016
:1029B00060042000C662020000000000F30F200047
:1029C0000300620044620200000000004822DE00B2
:1029D00003006200446202000000000020042000A6
:1029E000C662020000000000C00420004462020031
:1029F000000000009004200044620200000000007B
:102A00001005200044620200000000005005200074
:102A100044620200000000009004200044620200B2
:102A2000000000004004200044620200000000009A
:102A30000002200044620200000000006004200048
:102A400044620200000000005004200044620200C2
:102A50000000000020052000446202000000000089
:102A600040052000446202000000000090042000A5
:102A70004462020000000000C00420004462020022
:102A800000000000900420004462020000000000EA
:102A9000A005200044620200000000005004200055
:102AA0004462020000000000200520004462020091
:102AB000000000004426200060042000C6620200DE
:102AC00000000000F30F20000300620044620200D7
:102AD000000000004822DE000300620044620200A1
:102AE0000000000020042000C66202000000000078
:102AF00010042000446202000000000000052000D5
:102B00004462020000000000000520004462020050
:102B100000000000C0042000446202000000000029
:102B200090042000446202000000000030042000F5
:102B30004462020000000000100420004462020011
:102B40000000000040052000446202000000000078
:102B5000900420004462020000000000F004200005
:102B60004462020000000000E00420004462020011
:102B7000000000000002200044620200000000008B
:102B80000002200044620200000000005005200006
:102B90004462020000000000E004200044620200E1
:102BA00000000000900420004462020000000000C9
:102BB000400520004462020000000000C42D2000F7
:102BC00060042000C662020000000000F30F200035
:102BD0000300620044620200000000004822DE00A0
:102BE0000300620044620200000000002004200094
:102BF000C66202000000000070072000446202006C
:102C00000000000070072000446202000000000085
:102C1000700720004462020000000000E002200073
:102C2000446202000000000010062000446202001E
:102C30000000000070062000446202000000000056
:102C400020072000446202000000000090062000DF
:102C5000446202000000000070062000446202008E
:102C60000000000050062000446202000000000046
:102C7000C00620004462020000000000E0022000C4
:102C8000446202000000000030062000446202009E
:102C900000000000F0062000446202000000000076
:102CA000E00220004462020000000000A0072000B3
:102CB000446202000000000010062000446202008E
:102CC000000000003435200060042000C6620200CD
:102CD00000000000F30F20000300620044620200C5
:102CE000000000004822DE0003006200446202008F
:102CF0000000000020042000C66202000000000066
:102D00006005200044620200000000005006200020
:102D1000446202000000000020072000446202001C
:102D200000000000300720004462020000000000A4
:102D3000900620004462020000000000F00620001F
:102D40004462020000000000E0062000446202002D
:102D500000000000A0032000446202000000000008
:102D60000002200044620200000000005004200025
:102D700044620200000000002004200044620200BF
:102D80000000000000032000446202000000000078
:102D900080032000446202000000000000022000C6
:102DA000446202000000000010042000446202009F
:102DB00000000000C0062000446202000000000085
:102DC000000720004462020000000000800620008E
:102DD000446202000000000010062000446202006D
:102DE00000000000C435200060042000C66202001C
:102DF00000000000F30F20000300620044620200A4
:102E0000000000004822DE0003006200446202006D
:102E10000000000080BB2000E08288002230EC002F
:102E20008C0B0400000000005C10E2004220AF00A8
:102E30002230EC008C0B0400000000009E630200B6
:102E400000000000E411200060042000C6620200BF
:102E500000000000F30F2000030062004462020043
:102E6000000000004822DE0003006200446202000D
:102E70000000000020042000C662020000000000E4
:102E8000D004200044620200000000000002200084
:102E900044620200000000001004200044620200AE
:102EA0000000000000022000446202000000000058
:102EB0009004200044620200000000000002200094
:102EC0004462020000000000E004200044620200AE
:102ED0000000000000022000446202000000000028
:102EE00000022000446202000000000000022000F6
:102EF0004462020000000000D0042000446202008E
:102F000000000000000220004462020000000000F7
:102F10005004200044620200000000000002200073
:102F20004462020000000000E0042000446202004D
:102F300000000000000220004462020000000000C7
:102F400050052000446202000000000064142000CC
:102F500060042000C662020000000000F30F2000A1
:102F60000300620044620200000000004822DE000C
:102F70000300620044620200000000002004200000
:102F8000C662020000000000D0022000446202007D
:102F900000000000D0022000446202000000000097
:102FA000D00220004462020000000000D002200095
:102FB0004462020000000000D002200044620200CF
:102FC00000000000D0022000446202000000000067
:102FD000D00220004462020000000000D002200065
:102FE0004462020000000000D0022000446202009F
:102FF00000000000D0022000446202000000000037
:10300000D00220004462020000000000D002200034
:103010004462020000000000D0022000446202006E
:1030200000000000D0022000446202000000000006
:10303000D00220004462020000000000D002200004
:103040004462020000000000D0022000446202003E
:10305000000000000423200060042000C66202007B
:1030600000000000F30F2000030062004462020031
:10307000000000004822DE000300620044620200FB
:103080000000000020042000C662020000000000D2
:1030900040042000446202000000000010042000F0
:1030A000446202000000000040052000446202006B
:1030B0000000000010042000446202000000000034
:1030C0008425200060042000C66202000000000089
:1030D000F30F2000030062004462020000000000C1
:1030E0004822DE000300620044620200000000008B
:1030F00020042000C662020000000000D00420006E
:10310000446202000000000010042000446202003B
:1031100000000000E0042000446202000000000003
:10312000100420004462020000000000700420002F
:1031300044620200000000005004200044620200CB
:1031400000000000D00420004462020000000000E3
:10315000500420004462020000000000E00420004F
:1031600044620200000000004005200044620200AA
:1031700000000000843E200060042000C6620200BF
:1031800000000000F30F2000030062004462020010
:10319000000000004822DE000300620044620200DA
:1031A0000000000020042000C662020000000000B1
:1031B000300520004462020000000000500420009E
:1031C000446202000000000040052000446202004A
:1031D00000000000400520004462020000000000E2
:1031E000900420004462020000000000E00420007F
:1031F00044620200000000007004200044620200EB
:1032000000000000300520004462020000000000C1
:103210007409200060042000C66202000000000063
:10322000F30F20000300620044620200000000006F
:103230004822DE0003006200446202000000000039
:1032400020042000C66202000000000000052000EB
:103250004462020000000000C0042000446202003A
:103260000000000010042000446202000000000082
:10327000E00420004462020000000000400520003D
:10328000446202000000000090042000446202003A
:1032900000000000D0042000446202000000000092
:1032A000700420004462020000000000F40B2000C3
:1032B00060042000C662020000000000F30F20003E
:1032C0000300620044620200000000004822DE00A9
:1032D000030062004462020000000000200420009D
:1032E000C6620200000000003005200044620200B7
:1032F00000000000500420004462020000000000B2
:10330000400520004462020000000000400520004B
:1033100044620200000000009004200044620200A9
:1033200000000000E00420004462020000000000F1
:1033300070042000446202000000000030052000FC
:103340004462020000000000042520006004200008
:10335000C662020000000000F30F200003006200BC
:1033600044620200000000004822DE000300620008
:10337000446202000000000020042000C662020037
:103380000000000070052000446202000000000000
:10339000F00420004462020000000000200520002C
:1033A0004462020000000000B004200044620200F9
:1033B00000000000900420004462020000000000B1
:1033C000E0042000446202000000000070042000BD
:1033D0004462020000000000B427200060042000C6
:1033E000C662020000000000F30F2000030062002C
:1033F00044620200000000004822DE000300620078
:10340000446202000000000020042000C6620200A6
:1034100000000000D0042000446202000000000010
:10342000F00420004462020000000000400420007C
:1034300044620200000000005004200044620200C8
:10344000000000004440200060042000C66202002A
:1034500000000000F30F200003006200446202003D
:10346000000000004822DE00030062004462020007
:103470000000000020042000C662020000000000DE
:10348000300420004462020000000000100420000C
:103490004462020000000000C004200044620200F8
:1034A00000000000900420004462020000000000C0
:1034B00020042000446202000000000020052000DB
:1034C0004462020000000000100420004462020078
:1034D00000000000400520004462020000000000DF
:1034E000900420004462020000000000F00420006C
:1034F0004462020000000000E00420004462020078
:10350000000000003443200060042000C662020076
:1035100000000000F30F200003006200446202007C
:10352000000000004822DE00030062004462020046
:103530000000000020042000C6620200000000001D
:10354000D00420004462020000000000F0042000CB
:1035500044620200000000004004200044620200B7
:10356000000000005004200044620200000000003F
:103570008448200060042000C662020000000000B1
:10358000F30F20000300620044620200000000000C
:103590004822DE00030062004462020000000000D6
:1035A00020042000C6620200000000000005200088
:1035B0004462020000000000F004200044620200A7
:1035C00000000000700520004462020000000000BE
:1035D000500420004462020000000000200520008A
:1035E0004462020000000000000220004462020069
:1035F00000000000F004200044620200000000000F
:10360000600420004462020000000000600420000A
:10361000446202000000000080382100E08288003F
:103620002230EC008C0B04000000000090C68000EB
:1036300031002000010050004220AE002E1B04008B
:1036400000000000702102000000000020022000A5
:1036500010818800A61B04000000000090C68000B6
:1036600011002000010050004220AE00461B040063
:103670000000000070210200000000004000200057
:1036800010818800A61B04000000000090C6800086
:1036900021002000010050004220AE005A1B04000F
:1036A000000000006000200010818800A61B0400BC
:1036B0000000000090C68000910020000100500032
:1036C0004220AE006E1B04000000000080002000BD
:1036D00010818800A61B04000000000090C6800036
:1036E00081002000010050004220AE00821B040037
:1036F00000000000A000200010818800A61B04002C
:103700000000000090C68000710020000100500001
:103710004220AE00961B040000000000C000200004
:1037200010818800A61B0400000000005C10E2006D
:103730004220AE00A61B040000000000A0002000F4
:1037400010818800A61B0400000000008C0B040000
:10375000000000009E6302000000000084072000BB
:1037600060042000C662020000000000F30F200089
:103770000300620044620200000000004822DE00F4
:1037800003006200446202000000000020042000E8
:10379000C662020000000000100420004462020023
:1037A000000000000007200044620200000000004A
:1037B000000720004462020000000000C006200054
:1037C00044620200000000009006200044620200F3
:1037D000000000000423200060042000C6620200F4
:1037E00000000000F30F20000300620044620200AA
:1037F000000000004822DE00030062004462020074
:103800000000000020042000C6620200000000004A
:103810004004200044620200000000005006200026
:103820004462020000000000E00620004462020042
:103830000000000030072000446202000000000089
:10384000900620004462020000000000843E200038
:1038500060042000C662020000000000F30F200098
:103860000300620044620200000000004822DE0003
:1038700003006200446202000000000020042000F7
:10388000C662020000000000200520004462020021
:1038900000000000F006200044620200000000006A
:1038A000700720004462020000000000F0022000C7
:1038B0004462020000000000800420004462020014
:1038C00000000000B448200060042000C66202002E
:1038D00000000000F30F20000300620044620200B9
:1038E000000000004822DE00030062004462020083
:1038F0000000000020042000C6620200000000005A
:103900005449200060042000C6620200000000004C
:10391000F30F200003006200446202000000000078
:103920004822DE0003006200446202000000000042
:1039300020042000C662020000000000044A2000AB
:1039400060042000C662020000000000F30F2000A7
:103950000300620044620200000000004822DE0012
:103960000300620044620200000000002004200006
:10397000C662020000000000A44A2000600420008B
:10398000C662020000000000F30F20000300620086
:1039900044620200000000004822DE0003006200D2
:1039A000446202000000000020042000C662020001
:1039B00000000000F440200060042000C662020005
:1039C00000000000F30F20000300620044620200C8
:1039D000000000004822DE00030062004462020092
:1039E0000000000020042000C66202000000000069
:1039F00030052000446202000000000000072000A3
:103A000044620200000000005006200044620200F0
:103A10000000000050062000446202000000000088
:103A200040062000446202000000000074252000CF
:103A300060042000C662020000000000F30F2000B6
:103A40000300620044620200000000004822DE0021
:103A50000300620044620200000000002004200015
:103A6000C662020000000000300420004462020030
:103A70000000000010062000446202000000000068
:103A8000C0062000446202000000000090062000F2
:103A90004462020000000000200620004462020090
:103AA00000000000F409200060042000C66202004B
:103AB00000000000F30F20000300620044620200D7
:103AC000000000004822DE000300620044620200A1
:103AD0000000000020042000C66202000000000078
:103AE00030052000446202000000000000072000B2
:103AF0004462020000000000100620004462020040
:103B000000000000200720004462020000000000C6
:103B1000500620004462020000000000B44820006B
:103B200060042000C662020000000000F30F2000C5
:103B30000300620044620200000000004822DE0030
:103B4000030062004462020000000000D005200073
:103B5000C662020000000000400020004462020033
:103B6000000000007000200044620200000000001D
:103B700090052000C66202000000000070052000D1
:103B800044620200000000002230EC008C0B0400B4
:103B90000000000090828000808188005C67020045
:103BA00000000000B482800060042000C6620200B1
:103BB00000000000F30F20000300620044620200D6
:103BC000000000004822DE000300620044620200A0
:103BD0000000000020042000C66202000000000077
:103BE0005082800001032000010040004462020076
:103BF00000000000608280000103200001004000FE
:103C00004462020000000000708280000103200076
:103C10000100400044620200000000008082800039
:103C20000103200001004000446202000000000087
:103C3000B4828000C0828000000242006004200044
:103C4000C662020000000000F30F200003006200C3
:103C500044620200000000004822DE00030062000F
:103C6000446202000000000050828000D020020068
:103C700000000000508288005830EC006082800014
:103C8000D020020000000000608288005830EC0064
:103C900070828000D0200200000000007082880046
:103CA0005830EC0080828000D0200200000000002C
:103CB0008082880084828000A000200071828000C1
:103CC0000101B8000402410040062000618280002A
:103CD0000101B80004024100803E200051828000B2
:103CE0000101B8000402410094828800000006002F
:103CF00090828000808188005C67020000000000E4
:103D0000B482800060042000C6620200000000004F
:103D1000F30F200003006200446202000000000074
:103D20004822DE000300620044620200000000003E
:103D300020042000C66202000000000070828000A3
:103D40000103200001004000446202000000000066
:103D500080828000010320000100400044620200D4
:103D600000000000B4828000C08280000002420097
:103D700060042000C662020000000000F30F200073
:103D80000300620044620200000000004822DE00DE
:103D900003006200446202000000000070828000A4
:103DA000D020020000000000708288005830EC0033
:103DB00080828000D0200200000000008082880005
:103DC00084828000A0002000718280000101B80080
:103DD0000402410094828800000006009082800066
:103DE000808188005C67020000000000B4828000CF
:103DF00060042000C662020000000000F30F2000F3
:103E00000300620044620200000000004822DE005D
:103E10000300620044620200000000002004200051
:103E2000C6620200000000006082800001032000E2
:103E30000100400044620200000000007082800027
:103E40000103200001004000446202000000000065
:103E500080828000010320000100400044620200D3
:103E600000000000B4828000C08280000002420096
:103E700060042000C662020000000000F30F200072
:103E80000300620044620200000000004822DE00DD
:103E900003006200446202000000000060828000B3
:103EA000D020020000000000608288005830EC0042
:103EB00070828000D0200200000000007082880024
:103EC0005830EC0080828000D0200200000000000A
:103ED0008082880084828000A0002000718280009F
:103EE0000101B80004024100400620006182800008
:103EF0000101B8000402410094828800000006001D
:103F000090828000808188005C67020000000000D1
:103F1000B482800060042000C6620200000000003D
:103F2000F30F200003006200446202000000000062
:103F30004822DE000300620044620200000000002C
:103F400020042000C66202000000000050828000B1
:103F50000103200001004000446202000000000054
:103F600060828000010320000100400044620200E2
:103F7000000000007082800001032000010040006A
:103F800044620200000000008082800001032000E3
:103F9000010040004462020000000000B482800082
:103FA000C08280000002420060042000C66202005D
:103FB00000000000F30F20000300620044620200D2
:103FC000000000004822DE0003006200446202009C
:103FD0000000000050828000D0200200000000009D
:103FE000508288005830EC0060828000D0200200AF
:103FF00000000000608288005830EC007082800071
:10400000D020020000000000708288005830EC00D0
:1040100080828000D02002000000000080828800A2
:1040200084828000A0002000718280000101B8001D
:104030000402410040062000618280000101B800B6
:1040400004024100803E2000518280000101B8003E
:1040500004024100948288000000060090828000E3
:10406000808188005C67020000000000B48280004C
:1040700060042000C662020000000000F30F200070
:104080000300620044620200000000004822DE00DB
:1040900003006200446202000000000020042000CF
:1040A000C662020000000000508280000103200070
:1040B000010040004462020000000000E002200015
:1040C00044620200000000006082800001032000C2
:1040D0000100400044620200000000007082800085
:1040E00001032000010040004462020000000000C3
:1040F000B4828000C0828000000242006004200080
:10410000C662020000000000F30F200003006200FE
:1041100044620200000000004822DE00030062004A
:10412000446202000000000050828000D0200200A3
:1041300000000000508288005830EC005830EC003D
:1041400060828000D02002000000000060828800B1
:104150005830EC0070828000D02002000000000087
:104160007082880084828000A0002000718280001C
:104170000101B80004024100400620006182800075
:104180000101B80004024100803E200051828000FD
:104190000101B8000402410094828800000006007A
:1041A000D0828800B4828000C08280000002420079
:1041B00060042000C662020000000000F30F20002F
:1041C0000300620044620200000000004822DE009A
:1041D000030062004462020000000000200420008E
:1041E000C662020000000000D082800001032000AF
:1041F000010040004462020000000000B482800020
:10420000C08280000002420060042000C6620200FA
:1042100000000000F30F200003006200446202006F
:10422000000000004822DE00030062004462020039
:104230000000000090C680004100200001005000F6
:104240004220AE003A210400000000005A30EC0089
:10425000D0828000A1002000810050004200AF0009
:104260005A30EF007021020000000000D22004004C
:104270000000000090C680005100200001005000A6
:104280004220AE005C210400000000005A30ED0026
:10429000D0828000A1002000920020008100500008
:1042A0004200AF00D28288007021020000000000AE
:1042B000D22004000000000090C6800061002000B1
:1042C000010050004220AE001A210400000000004E
:1042D0007021020000000000D08280000000060073
:1042E00090C68000F1FF2F00010050004220AE0078
:1042F0007021040000000000000006009E63020020
:1043000000000000B407200060042000C662020024
:1043100000000000F30F200003006200446202006E
:10432000000000004822DE00030062004462020038
:104330000000000020042000C6620200000000000F
:10434000000520004462020000000000000220007E
:104350004462020000000000C00420004462020029
:104360000000000000022000446202000000000083
:10437000100420004462020000000000000220003F
:104380004462020000000000E004200044620200D9
:104390000000000000022000446202000000000053
:1043A00040052000446202000000000000022000DE
:1043B00044620200000000009004200044620200F9
:1043C0000000000000022000446202000000000023
:1043D000E00420004462020000000000000220000F
:1043E00044620200000000007004200044620200E9
:1043F00000000000000220004462020000000000F3
:1044000000022000446202000000000000022000C0
:1044100044620200000000003005200044620200F7
:1044200000000000000220004462020000000000C2
:10443000500420004462020000000000000220003E
:1044400044620200000000004005200044620200B7
:104450000000000000022000446202000000000092
:10446000400520004462020000000000000220001D
:104470004462020000000000900420004462020038
:104480000000000000022000446202000000000062
:10449000E00420004462020000000000000220004E
:1044A0004462020000000000700420004462020028
:1044B0000000000000022000446202000000000032
:1044C000300520004462020000000000340A200091
:1044D00060042000C662020000000000F30F20000C
:1044E0000300620044620200000000004822DE0077
:1044F000030062004462020000000000200420006B
:10450000C662020000000000D002200044620200E7
:1045100000000000D0022000446202000000000001
:10452000D00220004462020000000000D0022000FF
:104530004462020000000000D00220004462020039
:1045400000000000D00220004462020000000000D1
:10455000D00220004462020000000000D0022000CF
:104560004462020000000000D00220004462020009
:1045700000000000D00220004462020000000000A1
:10458000D00220004462020000000000D00220009F
:104590004462020000000000D002200044620200D9
:1045A00000000000D0022000446202000000000071
:1045B000D00220004462020000000000D00220006F
:1045C0004462020000000000D002200044620200A9
:1045D00000000000D0022000446202000000000041
:1045E000D00220004462020000000000D00220003F
:1045F0004462020000000000D00220004462020079
:1046000000000000D0022000446202000000000010
:10461000D00220004462020000000000D00220000E
:104620004462020000000000D00220004462020048
:1046300000000000D00220004462020000000000E0
:10464000D00220004462020000000000D0022000DE
:104650004462020000000000D00220004462020018
:1046600000000000D00220004462020000000000B0
:10467000D00220004462020000000000D0022000AE
:104680004462020000000000D002200044620200E8
:10469000000000000423200060042000C662020025
:1046A00000000000F30F20000300620044620200DB
:1046B000000000004822DE000300620044620200A5
:1046C0000000000020042000C6620200000000007C
:1046D00010838000808188005C6702000000000079
:1046E000608280000103200001004000446202005B
:1046F00000000000708280000103200001004000E3
:10470000446202000000000080828000010320005B
:10471000010040004462020000000000000220008E
:104720004462020000000000C00420004462020055
:10473000000000001004200044620200000000009D
:10474000E004200044620200000000004004200059
:1047500044620200000000000002200044620200E7
:1047600000000000E004200044620200000000009D
:10477000500520004462020000000000D004200028
:104780004462020000000000200420004462020095
:1047900000000000500420004462020000000000FD
:1047A000200520004462020000000000843E20003A
:1047B00060042000C662020000000000F30F200029
:1047C0000300620044620200000000004822DE0094
:1047D0000300620044620200000000002004200088
:1047E000C662020000000000900420004462020043
:1047F00000000000D004200044620200000000001D
:10480000000520004462020000000000C0042000F7
:1048100044620200000000005004200044620200D4
:1048200000000000D00420004462020000000000EC
:10483000500420004462020000000000E004200058
:1048400044620200000000004005200044620200B3
:10485000000000000441200060042000C662020045
:1048600000000000F30F2000030062004462020019
:10487000000000004822DE000300620044620200E3
:104880000000000020042000C662020000000000BA
:1048900030052000446202000000000050042000A7
:1048A0004462020000000000400520004462020053
:1048B00000000000400520004462020000000000EB
:1048C000900420004462020000000000E004200088
:1048D00044620200000000007004200044620200F4
:1048E00000000000300520004462020000000000CB
:1048F0008424200060042000C66202000000000042
:10490000F30F200003006200446202000000000078
:104910004822DE0003006200446202000000000042
:1049200020042000C6620200000000006004200095
:1049300044620200000000005004200044620200B3
:10494000000000002005200044620200000000007A
:104950004005200044620200000000009004200096
:104960004462020000000000C00420004462020013
:1049700000000000900420004462020000000000DB
:1049800030052000446202000000000050042000B6
:104990004462020000000000200520004462020082
:1049A000000000006427200060042000C6620200AE
:1049B00000000000F30F20000300620044620200C8
:1049C000000000004822DE00030062004462020092
:1049D0000000000020042000C66202000000000069
:1049E000B0062000446202000000000070062000B3
:1049F0004462020000000000F00220004462020055
:104A00000000000080062000446202000000000058
:104A100000022000446202000000000000838000C9
:104A2000808188005C6702000000000050828000E6
:104A30000103200001004000446202000000000069
:104A400060828000010320000100400044620200F7
:104A5000000000007082800001032000010040007F
:104A600044620200000000008082800001032000F8
:104A700001004000446202000000000004402000E9
:104A800060042000C662020000000000F30F200056
:104A90000300620044620200000000004822DE00C1
:104AA00003006200446202000000000020042000B5
:104AB000C6620200000000006004200044620200A0
:104AC00000000000500420004462020000000000CA
:104AD0002005200044620200000000004005200084
:104AE00044620200000000009004200044620200C2
:104AF00000000000C004200044620200000000002A
:104B000090042000446202000000000030052000F4
:104B100044620200000000005004200044620200D1
:104B20000000000020052000446202000000000098
:104B30000443200060042000C66202000000000060
:104B4000F30F200003006200446202000000000036
:104B50004822DE0003006200446202000000000000
:104B600020042000C6620200000000003005200082
:104B70004462020000000000700420004462020051
:104B8000000000000002200044620200000000005B
:104B9000F0808000808188005C67020000000000D7
:104BA00050828000010320000100400044620200A6
:104BB00000000000E002200044620200000000004B
:104BC0006082800001032000010040004462020076
:104BD00000000000708280000103200001004000FE
:104BE00044620200000000008448200060042000AD
:104BF000C662020000000000F30F20000300620004
:104C000044620200000000004822DE00030062004F
:104C1000446202000000000020042000C66202007E
:104C200000000000D00420004462020000000000E8
:104C300010042000446202000000000090042000E4
:104C40004462020000000000E00420004462020010
:104C5000000000000002200044620200000000008A
:104C6000D004200044620200000000005004200034
:104C70004462020000000000E004200044620200E0
:104C80000000000050052000446202000000000007
:104C90004449200060042000C662020000000000B9
:104CA000F30F2000030062004462020000000000D5
:104CB0004822DE000300620044620200000000009F
:104CC00020042000C66202000000000060042000F2
:104CD00044620200000000009004200044620200D0
:104CE00000000000200520004462020000000000D7
:104CF0003005200044620200000000004005200052
:104D00004462020000000000000220004462020031
:104D10000000000030052000446202000000000096
:104D2000500420004462020000000000C004200083
:104D300044620200000000005004200044620200AF
:104D40000000000030042000446202000000000067
:104D50004005200044620200000000000002200024
:104D6000446202000000000090042000446202003F
:104D70000000000040052000446202000000000026
:104D8000500420004462020000000000D004200013
:104D900044620200000000000002200044620200A1
:104DA00000000000400520004462020000000000F6
:104DB000F004200044620200000000000002200015
:104DC000446202000000000010042000446202005F
:104DD00000000000400420004462020000000000C7
:104DE000A0042000446202000000000050052000E2
:104DF000446202000000000030052000446202000E
:104E00000000000040052000446202000000000095
:104E100000712200E082880090002000108188004C
:104E20008C0B04000000000090C6800031002000C0
:104E3000010050004220AE00502704000000000096
:104E400070210200000000000071220080818800B3
:104E5000000020009081880000002000A0818800D0
:104E600040838000B081880000002000C08188005D
:104E700000002000D08188001E6F020000000000AA
:104E800080818000008188001C7802000000000002
:104E90002000200010818800C027040000000000CE
:104EA00090C6800011002000010050004220AE009A
:104EB00068270400000000007021020000000000CC
:104EC000E000200010818800C027040000000000DE
:104ED00090C6800021002000010050004220AE005A
:104EE0008027040000000000702102000000000084
:104EF0000001200010818800C0270400000000008D
:104F000090C6800081002000010050004220AE00C9
:104F1000982704000000000070210200000000003B
:104F20002001200010818800C0270400000000003C
:104F300090C6800071002000010050004220AE00A9
:104F4000B0270400000000007021020000000000F3
:104F50004001200010818800C027040000000000EC
:104F60005C10E2004220AE00C027040000000000F8
:104F70002000200010818800C027040000000000ED
:104F80008C0B040000000000844820006004200016
:104F9000C662020000000000F30F20000300620060
:104FA00044620200000000004822DE0003006200AC
:104FB000446202000000000020042000C6620200DB
:104FC0000000000000022000446202000000000017
:104FD00000022000446202000000000000022000E5
:104FE000446202000000000000022000446202004F
:104FF00000000000000220004462020000000000E7
:1050000000022000446202000000000000022000B4
:10501000446202000000000000022000446202001E
:1050200000000000000220004462020000000000B6
:105030004449200060042000C66202000000000015
:10504000F30F200003006200446202000000000031
:105050004822DE00030062004462020000000000FB
:1050600020042000C66202000000000000022000B0
:1050700044620200000000000002200044620200BE
:105080000000000050052000446202000000000003
:105090000005200044620200000000000002200021
:1050A000446202000000000000022000446202008E
:1050B0000000000000022000446202000000000026
:1050C00000022000446202000000000000022000F4
:1050D000446202000000000000022000446202005E
:1050E00000000000000220004462020000000000F6
:1050F0000002200044620200000000004004200082
:105100004462020000000000F0042000446202003B
:105110000000000070052000446202000000000052
:10512000E0042000446202000000000000022000B1
:1051300044620200000000000002200044620200FD
:105140000000000000022000446202000000000095
:105150000002200044620200000000000002200063
:1051600044620200000000000002200044620200CD
:105170000000000030052000446202000000000032
:10518000400520004462020000000000F0042000FE
:10519000446202000000000020052000446202007A
:1051A00000000000500420004462020000000000E3
:1051B000F0002000108188008C0B0400000000002B
:1051C000108380009082880000232000B082880035
:1051D00000002000C0828800EE1E020000000000D7
:1051E00090828000108388008448200060042000A2
:1051F000C662020000000000F30F200003006200FE
:1052000044620200000000004822DE000300620049
:10521000446202000000000020042000C662020078
:1052200000000000D00420004462020000000000E2
:1052300010042000446202000000000090042000DE
:105240004462020000000000E0042000446202000A
:105250000000000000022000446202000000000084
:10526000D00420004462020000000000500420002E
:105270004462020000000000E004200044620200DA
:105280000000000050052000446202000000000001
:105290004449200060042000C662020000000000B3
:1052A000F30F2000030062004462020000000000CF
:1052B0004822DE0003006200446202000000000099
:1052C00020042000C66202000000000060042000EC
:1052D00044620200000000009004200044620200CA
:1052E00000000000200520004462020000000000D1
:1052F000300520004462020000000000400520004C
:10530000446202000000000000022000446202002B
:105310000000000030052000446202000000000090
:10532000500420004462020000000000C00420007D
:1053300044620200000000005004200044620200A9
:105340000000000030042000446202000000000061
:10535000400520004462020000000000000220001E
:105360004462020000000000900420004462020039
:105370000000000040052000446202000000000020
:10538000500420004462020000000000D00420000D
:10539000446202000000000000022000446202009B
:1053A00000000000400520004462020000000000F0
:1053B000F00420004462020000000000000220000F
:1053C0004462020000000000100420004462020059
:1053D00000000000400420004462020000000000C1
:1053E000A0042000446202000000000050052000DC
:1053F0004462020000000000300520004462020008
:10540000000000004005200044620200000000008F
:1054100000712200E0828800900020001081880046
:105420008C0B040000000000844820006004200071
:10543000C662020000000000F30F200003006200BB
:1054400044620200000000004822DE000300620007
:10545000446202000000000020042000C662020036
:105460000000000000022000446202000000000072
:105470000002200044620200000000000002200040
:1054800044620200000000000002200044620200AA
:105490000000000000022000446202000000000042
:1054A0000002200044620200000000000002200010
:1054B000446202000000000000022000446202007A
:1054C0000000000000022000446202000000000012
:1054D0004449200060042000C66202000000000071
:1054E000F30F20000300620044620200000000008D
:1054F0004822DE0003006200446202000000000057
:1055000020042000C662020000000000000220000B
:105510004462020000000000000220004462020019
:10552000000000005005200044620200000000005E
:10553000000520004462020000000000000220007C
:1055400044620200000000000002200044620200E9
:105550000000000000022000446202000000000081
:10556000000220004462020000000000000220004F
:1055700044620200000000000002200044620200B9
:105580000000000000022000446202000000000051
:1055900000022000446202000000000040042000DD
:1055A0004462020000000000F00420004462020097
:1055B00000000000700520004462020000000000AE
:1055C000E00420004462020000000000000220000D
:1055D0004462020000000000000220004462020059
:1055E00000000000000220004462020000000000F1
:1055F00000022000446202000000000000022000BF
:105600004462020000000000000220004462020028
:10561000000000003005200044620200000000008D
:10562000400520004462020000000000F004200059
:1056300044620200000000002005200044620200D5
:10564000000000005004200044620200000000003E
:1056500030012000108188008C0B04000000000045
:105660000083800090828800B0272000B0828800EC
:1056700000002000C0828800801F0200000000009F
:10568000908280000083880084482000600420000D
:10569000C662020000000000F30F20000300620059
:1056A00044620200000000004822DE0003006200A5
:1056B000446202000000000020042000C6620200D4
:1056C00000000000D004200044620200000000003E
:1056D000100420004462020000000000900420003A
:1056E0004462020000000000E00420004462020066
:1056F00000000000000220004462020000000000E0
:10570000D004200044620200000000005004200089
:105710004462020000000000E00420004462020035
:10572000000000005005200044620200000000005C
:105730004449200060042000C6620200000000000E
:10574000F30F20000300620044620200000000002A
:105750004822DE00030062004462020000000000F4
:1057600020042000C6620200000000006004200047
:105770004462020000000000900420004462020025
:10578000000000002005200044620200000000002C
:1057900030052000446202000000000040052000A7
:1057A0004462020000000000000220004462020087
:1057B00000000000300520004462020000000000EC
:1057C000500420004462020000000000C0042000D9
:1057D0004462020000000000500420004462020005
:1057E00000000000300420004462020000000000BD
:1057F000400520004462020000000000000220007A
:105800004462020000000000900420004462020094
:10581000000000004005200044620200000000007B
:10582000500420004462020000000000D004200068
:1058300044620200000000000002200044620200F6
:10584000000000004005200044620200000000004B
:10585000F00420004462020000000000000220006A
:1058600044620200000000001004200044620200B4
:10587000000000004004200044620200000000001C
:10588000A004200044620200000000005005200037
:105890004462020000000000300520004462020063
:1058A00000000000400520004462020000000000EB
:1058B00000712200E08288009000200010818800A2
:1058C0008C0B0400000000008448200060042000CD
:1058D000C662020000000000F30F20000300620017
:1058E00044620200000000004822DE000300620063
:1058F000446202000000000020042000C662020092
:1059000000000000000220004462020000000000CD
:10591000000220004462020000000000000220009B
:105920004462020000000000000220004462020005
:10593000000000000002200044620200000000009D
:10594000000220004462020000000000000220006B
:1059500044620200000000000002200044620200D5
:10596000000000000002200044620200000000006D
:105970004449200060042000C662020000000000CC
:10598000F30F2000030062004462020000000000E8
:105990004822DE00030062004462020000000000B2
:1059A00020042000C6620200000000000002200067
:1059B0004462020000000000000220004462020075
:1059C00000000000500520004462020000000000BA
:1059D00000052000446202000000000000022000D8
:1059E0004462020000000000000220004462020045
:1059F00000000000000220004462020000000000DD
:105A000000022000446202000000000000022000AA
:105A10004462020000000000000220004462020014
:105A200000000000000220004462020000000000AC
:105A30000002200044620200000000004004200038
:105A40004462020000000000F004200044620200F2
:105A50000000000070052000446202000000000009
:105A6000E004200044620200000000000002200068
:105A700044620200000000000002200044620200B4
:105A8000000000000002200044620200000000004C
:105A9000000220004462020000000000000220001A
:105AA0004462020000000000000220004462020084
:105AB00000000000300520004462020000000000E9
:105AC000400520004462020000000000F0042000B5
:105AD0004462020000000000200520004462020031
:105AE000000000005004200044620200000000009A
:105AF00050012000108188008C0B04000000000081
:105B0000F08080009082880030432000B0828800BE
:105B100000002000C08288002E200200000000004B
:105B200090828000F080880084482000600420007B
:105B3000C662020000000000F30F200003006200B4
:105B400044620200000000004822DE000300620000
:105B5000446202000000000020042000C66202002F
:105B600000000000D0042000446202000000000099
:105B70001004200044620200000000009004200095
:105B80004462020000000000E004200044620200C1
:105B9000000000000002200044620200000000003B
:105BA000D0042000446202000000000050042000E5
:105BB0004462020000000000E00420004462020091
:105BC00000000000500520004462020000000000B8
:105BD0004449200060042000C6620200000000006A
:105BE000F30F200003006200446202000000000086
:105BF0004822DE0003006200446202000000000050
:105C000020042000C66202000000000060042000A2
:105C10004462020000000000900420004462020080
:105C20000000000020052000446202000000000087
:105C30003005200044620200000000004005200002
:105C400044620200000000000002200044620200E2
:105C50000000000030052000446202000000000047
:105C6000500420004462020000000000C004200034
:105C70004462020000000000500420004462020060
:105C80000000000030042000446202000000000018
:105C900040052000446202000000000000022000D5
:105CA00044620200000000009004200044620200F0
:105CB00000000000400520004462020000000000D7
:105CC000500420004462020000000000D0042000C4
:105CD0004462020000000000000220004462020052
:105CE00000000000400520004462020000000000A7
:105CF000F0042000446202000000000000022000C6
:105D0000446202000000000010042000446202000F
:105D10000000000040042000446202000000000077
:105D2000A004200044620200000000005005200092
:105D300044620200000000003005200044620200BE
:105D40000000000040052000446202000000000046
:105D500000712200E08288009000200010818800FD
:105D60008C0B0400000000009E6302000000000095
:105D7000B408200060042000C66202000000000099
:105D8000F30F2000030062004462020000000000E4
:105D90004822DE00030062004462020000000000AE
:105DA00020042000C66202000000000090042000D1
:105DB0004462020000000000000220004462020071
:105DC00000000000D0042000446202000000000037
:105DD00000022000446202000000000000052000D4
:105DE0004462020000000000000220004462020041
:105DF00000000000C0042000446202000000000017
:105E00000002200044620200000000005004200054
:105E10004462020000000000000220004462020010
:105E200000000000D00420004462020000000000D6
:105E30000002200044620200000000005004200024
:105E400044620200000000000002200044620200E0
:105E500000000000E0042000446202000000000096
:105E60000002200044620200000000004005200003
:105E70004462020000000000340B20006004200097
:105E8000C662020000000000F30F20000300620061
:105E900044620200000000004822DE0003006200AD
:105EA000446202000000000020042000C6620200DC
:105EB00000000000D0022000446202000000000048
:105EC000D00220004462020000000000D002200046
:105ED0004462020000000000D00220004462020080
:105EE00000000000D0022000446202000000000018
:105EF000D00220004462020000000000D002200016
:105F00004462020000000000D0022000446202004F
:105F100000000000D00220004462020000000000E7
:105F2000D00220004462020000000000D0022000E5
:105F30004462020000000000D0022000446202001F
:105F400000000000D00220004462020000000000B7
:105F5000D00220004462020000000000D0022000B5
:105F60004462020000000000D002200044620200EF
:105F700000000000D0022000446202000000000087
:105F80004410200060042000C662020000000000EF
:105F9000F30F2000030062004462020000000000D2
:105FA0004822DE000300620044620200000000009C
:105FB00020042000C662020000000000300520001E
:105FC000446202000000000000022000446202005F
:105FD00000000000500420004462020000000000A5
:105FE0000002200044620200000000004005200082
:105FF000446202000000000000022000446202002F
:106000000000000040052000446202000000000083
:106010000002200044620200000000009004200002
:1060200044620200000000000002200044620200FE
:1060300000000000E00420004462020000000000B4
:1060400000022000446202000000000070042000F2
:1060500044620200000000000002200044620200CE
:106060000000000030052000446202000000000033
:10607000C412200060042000C6620200000000007C
:10608000F30F2000030062004462020000000000E1
:106090004822DE00030062004462020000000000AB
:1060A00020042000C662020000000000D002200090
:1060B0004462020000000000D0022000446202009E
:1060C00000000000D0022000446202000000000036
:1060D000D00220004462020000000000D002200034
:1060E0004462020000000000D0022000446202006E
:1060F00000000000D0022000446202000000000006
:10610000D00220004462020000000000D002200003
:106110004462020000000000D0022000446202003D
:1061200000000000D00220004462020000000000D5
:10613000D00220004462020000000000D0022000D3
:106140004462020000000000D0022000446202000D
:1061500000000000D00220004462020000000000A5
:106160008407200060042000C662020000000000D6
:10617000F30F2000030062004462020000000000F0
:106180004822DE00030062004462020000000000BA
:1061900020042000C662020000000000208380006E
:1061A000808188005C67020000000000708280002F
:1061B00001032000010040004462020000000000D2
:1061C0008082800001032000010040004462020040
:1061D00000000000000220004462020000000000F5
:1061E000900420004462020000000000E002200051
:1061F00044620200000000004004200044620200EB
:1062000000000000E00220004462020000000000E4
:10621000000220004462020000000000E0042000B0
:106220004462020000000000F00620004462020008
:10623000000000000423200060042000C662020069
:1062400000000000F30F200003006200446202001F
:10625000000000004822DE000300620044620200E9
:106260000000000020042000C662020000000000C0
:1062700030838000808188005C670200000000009D
:10628000708280000103200001004000446202008F
:106290000000000080828000010320000100400017
:1062A000446202000000000000022000446202007C
:1062B00000000000E0042000446202000000000032
:1062C000F0062000446202000000000000022000EE
:1062D0004462020000000000F0042000446202005A
:1062E0000000000060042000446202000000000082
:1062F000000220004462020000000000200520008F
:106300004462020000000000F00420004462020029
:106310000000000070052000446202000000000040
:10632000300520004462020000000000843E20008E
:1063300060042000C662020000000000F30F20008D
:106340000300620044620200000000004822DE00F8
:1063500003006200446202000000000020042000EC
:10636000C662020000000000408380008081880037
:106370005C670200000000006082800001032000D2
:1063800001004000446202000000000070828000B2
:1063900001032000010040004462020000000000F0
:1063A000808280000103200001004000446202005E
:1063B0000000000000022000446202000000000013
:1063C000200520004462020000000000F0042000CC
:1063D00044620200000000007005200044620200D8
:1063E00000000000000220004462020000000000E3
:1063F00070052000446202000000000090042000AC
:1064000044620200000000004004200044620200D8
:10641000000000004005200044620200000000006F
:1064200080042000446202000000000000022000FE
:1064300044620200000000003006200044620200B6
:1064400000000000D00620004462020000000000AE
:106450001424200060042000C66202000000000036
:10646000F30F2000030062004462020000000000FD
:106470004822DE00030062004462020000000000C7
:1064800020042000C6620200000000000005200079
:106490004462020000000000C004200044620200C8
:1064A0000000000010042000446202000000000010
:1064B000E0042000446202000000000040052000CB
:1064C0004462020000000000500420004462020008
:1064D00000000000200520004462020000000000CF
:1064E000000220004462020000000000F0022000D0
:1064F000446202000000000000022000446202002A
:10650000000000003004200044620200000000008F
:10651000500520004462020000000000C00420007A
:1065200044620200000000004005200044620200B6
:1065300000000000900420004462020000000000FF
:1065400060052000446202000000000010042000EA
:106550004462020000000000400520004462020086
:1065600000000000F004200044620200000000006F
:10657000200520004462020000000000000220000C
:106580004462020000000000508380004462020068
:1065900000000000D43F200060042000C66202001A
:1065A00000000000F30F20000300620044620200BC
:1065B000000000004822DE00030062004462020086
:1065C0000000000020042000C6620200000000005D
:1065D000400520004462020000000000100420007A
:1065E0004462020000000000E00420004462020057
:1065F00000000000B004200044620200000000001F
:10660000000220004462020000000000300420006C
:1066100044620200000000001004200044620200F6
:10662000000000000005200044620200000000009D
:10663000100420004462020000000000300420002A
:106640004462020000000000900420004462020046
:10665000000000004005200044620200000000002D
:1066600090052000446202000000000000022000AB
:106670004462020000000000C442200060042000C8
:10668000C662020000000000F30F20000300620059
:1066900044620200000000004822DE0003006200A5
:1066A000446202000000000020042000C6620200D4
:1066B00000000000C004200044620200000000004E
:1066C0009004200044620200000000004005200009
:1066D0004462020000000000200520004462020025
:1066E000000000005004200044620200000000008E
:1066F000300520004462020000000000000220007B
:1067000044620200000000006083800080818800F5
:106710005C6702000000000050828000010320003E
:10672000010040004462020000000000608280001E
:10673000010320000100400044620200000000004C
:1067400070828000010320000100400044620200CA
:106750000000000080828000010320000100400052
:106760004462020000000000844820006004200011
:10677000C662020000000000F30F20000300620068
:1067800044620200000000004822DE0003006200B4
:10679000446202000000000020042000C6620200E3
:1067A000000000000002200044620200000000001F
:1067B00000022000446202000000000000022000ED
:1067C0004462020000000000200420004462020035
:1067D00000000000100420004462020000000000DD
:1067E000300420004462020000000000B0042000D9
:1067F0004462020000000000000220004462020027
:1068000000000000000220004462020000000000BE
:106810004449200060042000C6620200000000001D
:10682000F30F200003006200446202000000000039
:106830004822DE0003006200446202000000000003
:1068400020042000C6620200000000006004200056
:106850004462020000000000900420004462020034
:10686000000000002005200044620200000000003B
:1068700030052000446202000000000040052000B6
:106880004462020000000000000220004462020096
:1068900000000000300520004462020000000000FB
:1068A000500420004462020000000000C0042000E8
:1068B0004462020000000000500420004462020014
:1068C00000000000300420004462020000000000CC
:1068D0004005200044620200000000000002200089
:1068E00044620200000000009004200044620200A4
:1068F000000000004005200044620200000000008B
:10690000500420004462020000000000D004200077
:106910004462020000000000000220004462020005
:10692000000000004005200044620200000000005A
:10693000F004200044620200000000000002200079
:1069400044620200000000001004200044620200C3
:10695000000000004004200044620200000000002B
:10696000A004200044620200000000005005200046
:106970004462020000000000300520004462020072
:1069800000000000400520004462020000000000FA
:1069900000712200E0828800100120001081880030
:1069A0008C0B04000000000090C680003100200025
:1069B000010050004220AE00EC3404000000000052
:1069C000702102000000000080002000108188007B
:1069D000743504000000000090C680000100200013
:1069E000010050004220AE00043504000000000009
:1069F000702102000000000060012000108188006A
:106A0000743504000000000090C6800011002000D2
:106A1000010050004220AE001C35040000000000C0
:106A20007021020000000000800120001081880019
:106A3000743504000000000090C680002100200092
:106A4000010050004220AE00343504000000000078
:106A50007021020000000000A001200010818800C9
:106A6000743504000000000090C680008100200002
:106A7000010050004220AE004C3504000000000030
:106A80007021020000000000C00120001081880079
:106A9000743504000000000090C6800071002000E2
:106AA000010050004220AE006435040000000000E8
:106AB0007021020000000000E00120001081880029
:106AC00074350400000000005C10E2004220AE00BB
:106AD0007435040000000000800020001081880050
:106AE00074350400000000008C0B0400000000005E
:106AF0008448200060042000C662020000000000FC
:106B0000F30F200003006200446202000000000056
:106B10004822DE0003006200446202000000000020
:106B200020042000C66202000000000000022000D5
:106B300044620200000000000002200044620200E3
:106B4000000000000002200044620200000000007B
:106B50000002200044620200000000000002200049
:106B600044620200000000000002200044620200B3
:106B7000000000000002200044620200000000004B
:106B80000002200044620200000000000002200019
:106B9000446202000000000044492000600420001C
:106BA000C662020000000000F30F20000300620034
:106BB00044620200000000004822DE000300620080
:106BC000446202000000000020042000C6620200AF
:106BD00000000000000220004462020000000000EB
:106BE0000002200044620200000000005005200066
:106BF0004462020000000000000520004462020020
:106C000000000000000220004462020000000000BA
:106C10000002200044620200000000000002200088
:106C200044620200000000000002200044620200F2
:106C3000000000000002200044620200000000008A
:106C40000002200044620200000000000002200058
:106C500044620200000000000002200044620200C2
:106C60000000000040042000446202000000000018
:106C7000F0042000446202000000000070052000C3
:106C80004462020000000000E004200044620200B0
:106C9000000000000002200044620200000000002A
:106CA00000022000446202000000000000022000F8
:106CB0004462020000000000000220004462020062
:106CC00000000000000220004462020000000000FA
:106CD0000002200044620200000000003005200095
:106CE00044620200000000004005200044620200EF
:106CF00000000000F00420004462020000000000D8
:106D00002005200044620200000000005004200022
:106D10004462020000000000700120001081880021
:106D20008C0B04000000000020838000908288000B
:106D300080072000B082880000002000C082880008
:106D4000781E0200000000009082800020838800EE
:106D50008448200060042000C66202000000000099
:106D6000F30F2000030062004462020000000000F4
:106D70004822DE00030062004462020000000000BE
:106D800020042000C6620200000000000002200073
:106D90004462020000000000000220004462020081
:106DA0000000000000022000446202000000000019
:106DB00020042000446202000000000010042000B3
:106DC000446202000000000030042000446202001F
:106DD00000000000B0042000446202000000000037
:106DE00000022000446202000000000000022000B7
:106DF00044620200000000004449200060042000BA
:106E0000C662020000000000F30F200003006200D1
:106E100044620200000000004822DE00030062001D
:106E2000446202000000000020042000C66202004C
:106E30000000000060042000446202000000000026
:106E400090042000446202000000000020052000A1
:106E5000446202000000000030052000446202008D
:106E60000000000040052000446202000000000015
:106E700000022000446202000000000030052000F3
:106E8000446202000000000050042000446202003E
:106E900000000000C0042000446202000000000066
:106EA0005004200044620200000000003004200072
:106EB000446202000000000040052000446202001D
:106EC00000000000000220004462020000000000F8
:106ED00090042000446202000000000040052000F1
:106EE00044620200000000005004200044620200DE
:106EF00000000000D00420004462020000000000F6
:106F00000002200044620200000000004005200052
:106F10004462020000000000F0042000446202000D
:106F20000000000000022000446202000000000097
:106F30001004200044620200000000004004200011
:106F40004462020000000000A0042000446202002D
:106F50000000000050052000446202000000000014
:106F600030052000446202000000000040052000BF
:106F7000446202000000000000712200E0828800EC
:106F800010012000108188008C0B0400000000001C
:106F90008448200060042000C66202000000000057
:106FA000F30F2000030062004462020000000000B2
:106FB0004822DE000300620044620200000000007C
:106FC00020042000C6620200000000000002200031
:106FD000446202000000000000022000446202003F
:106FE00000000000000220004462020000000000D7
:106FF00000022000446202000000000000022000A5
:10700000446202000000000000022000446202000E
:1070100000000000000220004462020000000000A6
:107020000002200044620200000000000002200074
:107030004462020000000000444920006004200077
:10704000C662020000000000F30F2000030062008F
:1070500044620200000000004822DE0003006200DB
:10706000446202000000000020042000C66202000A
:107070000000000000022000446202000000000046
:1070800000022000446202000000000050052000C1
:10709000446202000000000000052000446202007B
:1070A0000000000000022000446202000000000016
:1070B00000022000446202000000000000022000E4
:1070C000446202000000000000022000446202004E
:1070D00000000000000220004462020000000000E6
:1070E00000022000446202000000000000022000B4
:1070F000446202000000000000022000446202001E
:107100000000000040042000446202000000000073
:10711000F00420004462020000000000700520001E
:107120004462020000000000E0042000446202000B
:107130000000000000022000446202000000000085
:107140000002200044620200000000000002200053
:1071500044620200000000000002200044620200BD
:107160000000000000022000446202000000000055
:1071700000022000446202000000000030052000F0
:10718000446202000000000040052000446202004A
:1071900000000000F0042000446202000000000033
:1071A000200520004462020000000000500420007E
:1071B000446202000000000090012000108188005D
:1071C0008C0B040000000000308380009082880057
:1071D00000232000B082880000002000C0828800C8
:1071E000781E02000000000090828000308388003A
:1071F0008448200060042000C662020000000000F5
:10720000F30F20000300620044620200000000004F
:107210004822DE0003006200446202000000000019
:1072200020042000C66202000000000000022000CE
:1072300044620200000000000002200044620200DC
:107240000000000000022000446202000000000074
:10725000200420004462020000000000100420000E
:10726000446202000000000030042000446202007A
:1072700000000000B0042000446202000000000092
:107280000002200044620200000000000002200012
:107290004462020000000000444920006004200015
:1072A000C662020000000000F30F2000030062002D
:1072B00044620200000000004822DE000300620079
:1072C000446202000000000020042000C6620200A8
:1072D0000000000060042000446202000000000082
:1072E00090042000446202000000000020052000FD
:1072F00044620200000000003005200044620200E9
:107300000000000040052000446202000000000070
:10731000000220004462020000000000300520004E
:107320004462020000000000500420004462020099
:1073300000000000C00420004462020000000000C1
:1073400050042000446202000000000030042000CD
:107350004462020000000000400520004462020078
:107360000000000000022000446202000000000053
:10737000900420004462020000000000400520004C
:107380004462020000000000500420004462020039
:1073900000000000D0042000446202000000000051
:1073A00000022000446202000000000040052000AE
:1073B0004462020000000000F00420004462020069
:1073C00000000000000220004462020000000000F3
:1073D000100420004462020000000000400420006D
:1073E0004462020000000000A00420004462020089
:1073F0000000000050052000446202000000000070
:10740000300520004462020000000000400520001A
:10741000446202000000000000712200E082880047
:1074200010012000108188008C0B04000000000077
:107430008448200060042000C662020000000000B2
:10744000F30F20000300620044620200000000000D
:107450004822DE00030062004462020000000000D7
:1074600020042000C662020000000000000220008C
:10747000446202000000000000022000446202009A
:107480000000000000022000446202000000000032
:107490000002200044620200000000000002200000
:1074A000446202000000000000022000446202006A
:1074B0000000000000022000446202000000000002
:1074C00000022000446202000000000000022000D0
:1074D00044620200000000004449200060042000D3
:1074E000C662020000000000F30F200003006200EB
:1074F00044620200000000004822DE000300620037
:10750000446202000000000020042000C662020065
:1075100000000000000220004462020000000000A1
:10752000000220004462020000000000500520001C
:1075300044620200000000000005200044620200D6
:107540000000000000022000446202000000000071
:10755000000220004462020000000000000220003F
:1075600044620200000000000002200044620200A9
:107570000000000000022000446202000000000041
:10758000000220004462020000000000000220000F
:107590004462020000000000000220004462020079
:1075A00000000000400420004462020000000000CF
:1075B000F00420004462020000000000700520007A
:1075C0004462020000000000E00420004462020067
:1075D00000000000000220004462020000000000E1
:1075E00000022000446202000000000000022000AF
:1075F0004462020000000000000220004462020019
:1076000000000000000220004462020000000000B0
:10761000000220004462020000000000300520004B
:1076200044620200000000004005200044620200A5
:1076300000000000F004200044620200000000008E
:1076400020052000446202000000000050042000D9
:107650004462020000000000B00120001081880098
:107660008C0B0400000000004083800090828800A2
:10767000803E2000B082880000002000C082880088
:10768000EE1E02000000000090828000408388000F
:107690008448200060042000C66202000000000050
:1076A000F30F2000030062004462020000000000AB
:1076B0004822DE0003006200446202000000000075
:1076C00020042000C662020000000000000220002A
:1076D0004462020000000000000220004462020038
:1076E00000000000000220004462020000000000D0
:1076F000200420004462020000000000100420006A
:1077000044620200000000003004200044620200D5
:1077100000000000B00420004462020000000000ED
:10772000000220004462020000000000000220006D
:107730004462020000000000444920006004200070
:10774000C662020000000000F30F20000300620088
:1077500044620200000000004822DE0003006200D4
:10776000446202000000000020042000C662020003
:1077700000000000600420004462020000000000DD
:107780009004200044620200000000002005200058
:107790004462020000000000300520004462020044
:1077A00000000000400520004462020000000000CC
:1077B00000022000446202000000000030052000AA
:1077C00044620200000000005004200044620200F5
:1077D00000000000C004200044620200000000001D
:1077E0005004200044620200000000003004200029
:1077F00044620200000000004005200044620200D4
:1078000000000000000220004462020000000000AE
:1078100090042000446202000000000040052000A7
:107820004462020000000000500420004462020094
:1078300000000000D00420004462020000000000AC
:107840000002200044620200000000004005200009
:107850004462020000000000F004200044620200C4
:10786000000000000002200044620200000000004E
:1078700010042000446202000000000040042000C8
:107880004462020000000000A004200044620200E4
:1078900000000000500520004462020000000000CB
:1078A0003005200044620200000000004005200076
:1078B000446202000000000000712200E0828800A3
:1078C00010012000108188008C0B040000000000D3
:1078D0008448200060042000C6620200000000000E
:1078E000F30F200003006200446202000000000069
:1078F0004822DE0003006200446202000000000033
:1079000020042000C66202000000000000022000E7
:1079100044620200000000000002200044620200F5
:10792000000000000002200044620200000000008D
:10793000000220004462020000000000000220005B
:1079400044620200000000000002200044620200C5
:10795000000000000002200044620200000000005D
:10796000000220004462020000000000000220002B
:10797000446202000000000044492000600420002E
:10798000C662020000000000F30F20000300620046
:1079900044620200000000004822DE000300620092
:1079A000446202000000000020042000C6620200C1
:1079B00000000000000220004462020000000000FD
:1079C0000002200044620200000000005005200078
:1079D0004462020000000000000520004462020032
:1079E00000000000000220004462020000000000CD
:1079F000000220004462020000000000000220009B
:107A00004462020000000000000220004462020004
:107A1000000000000002200044620200000000009C
:107A2000000220004462020000000000000220006A
:107A300044620200000000000002200044620200D4
:107A4000000000004004200044620200000000002A
:107A5000F0042000446202000000000070052000D5
:107A60004462020000000000E004200044620200C2
:107A7000000000000002200044620200000000003C
:107A8000000220004462020000000000000220000A
:107A90004462020000000000000220004462020074
:107AA000000000000002200044620200000000000C
:107AB00000022000446202000000000030052000A7
:107AC0004462020000000000400520004462020001
:107AD00000000000F00420004462020000000000EA
:107AE0002005200044620200000000005004200035
:107AF0004462020000000000D001200010818800D4
:107B00008C0B04000000000084482000600420006A
:107B1000C662020000000000F30F200003006200B4
:107B200044620200000000004822DE000300620000
:107B3000446202000000000020042000C66202002F
:107B4000000000000002200044620200000000006B
:107B50000002200044620200000000000002200039
:107B60004462020000000000200420004462020081
:107B70000000000010042000446202000000000029
:107B8000300420004462020000000000B004200025
:107B90004462020000000000000220004462020073
:107BA000000000000002200044620200000000000B
:107BB0004449200060042000C6620200000000006A
:107BC000F30F200003006200446202000000000086
:107BD0004822DE0003006200446202000000000050
:107BE00020042000C66202000000000060042000A3
:107BF0004462020000000000900420004462020081
:107C00000000000020052000446202000000000087
:107C10003005200044620200000000004005200002
:107C200044620200000000000002200044620200E2
:107C30000000000030052000446202000000000047
:107C4000500420004462020000000000C004200034
:107C50004462020000000000500420004462020060
:107C60000000000030042000446202000000000018
:107C700040052000446202000000000000022000D5
:107C800044620200000000009004200044620200F0
:107C900000000000400520004462020000000000D7
:107CA000500420004462020000000000D0042000C4
:107CB0004462020000000000000220004462020052
:107CC00000000000400520004462020000000000A7
:107CD000F0042000446202000000000000022000C6
:107CE0004462020000000000100420004462020010
:107CF0000000000040042000446202000000000078
:107D0000A004200044620200000000005005200092
:107D100044620200000000003005200044620200BE
:107D20000000000040052000446202000000000046
:107D300000712200E082880010012000108188007C
:107D40008C0B040000000000844820006004200028
:107D5000C662020000000000F30F20000300620072
:107D600044620200000000004822DE0003006200BE
:107D7000446202000000000020042000C6620200ED
:107D80000000000000022000446202000000000029
:107D900000022000446202000000000000022000F7
:107DA0004462020000000000000220004462020061
:107DB00000000000000220004462020000000000F9
:107DC00000022000446202000000000000022000C7
:107DD0004462020000000000000220004462020031
:107DE00000000000000220004462020000000000C9
:107DF0004449200060042000C66202000000000028
:107E0000F30F200003006200446202000000000043
:107E10004822DE000300620044620200000000000D
:107E200020042000C66202000000000000022000C2
:107E300044620200000000000002200044620200D0
:107E40000000000050052000446202000000000015
:107E50000005200044620200000000000002200033
:107E600044620200000000000002200044620200A0
:107E70000000000000022000446202000000000038
:107E80000002200044620200000000000002200006
:107E90004462020000000000000220004462020070
:107EA0000000000000022000446202000000000008
:107EB0000002200044620200000000004004200094
:107EC0004462020000000000F0042000446202004E
:107ED0000000000070052000446202000000000065
:107EE000E0042000446202000000000000022000C4
:107EF0004462020000000000000220004462020010
:107F000000000000000220004462020000000000A7
:107F10000002200044620200000000000002200075
:107F200044620200000000000002200044620200DF
:107F30000000000030052000446202000000000044
:107F4000400520004462020000000000F004200010
:107F5000446202000000000020052000446202008C
:107F600000000000500420004462020000000000F5
:107F7000F0012000108188008C0B0400000000003C
:107F8000608380009082880030432000B0828800A7
:107F900000002000C0828800801F02000000000056
:107FA0009082800060838800844820006004200064
:107FB000C662020000000000F30F20000300620010
:107FC00044620200000000004822DE00030062005C
:107FD000446202000000000020042000C66202008B
:107FE00000000000000220004462020000000000C7
:107FF0000002200044620200000000000002200095
:1080000044620200000000002004200044620200DC
:108010000000000010042000446202000000000084
:10802000300420004462020000000000B004200080
:1080300044620200000000000002200044620200CE
:108040000000000000022000446202000000000066
:108050004449200060042000C662020000000000C5
:10806000F30F2000030062004462020000000000E1
:108070004822DE00030062004462020000000000AB
:1080800020042000C66202000000000060042000FE
:1080900044620200000000009004200044620200DC
:1080A00000000000200520004462020000000000E3
:1080B000300520004462020000000000400520005E
:1080C000446202000000000000022000446202003E
:1080D00000000000300520004462020000000000A3
:1080E000500420004462020000000000C004200090
:1080F00044620200000000005004200044620200BC
:108100000000000030042000446202000000000073
:108110004005200044620200000000000002200030
:10812000446202000000000090042000446202004B
:108130000000000040052000446202000000000032
:10814000500420004462020000000000D00420001F
:1081500044620200000000000002200044620200AD
:108160000000000040052000446202000000000002
:10817000F004200044620200000000000002200021
:10818000446202000000000010042000446202006B
:1081900000000000400420004462020000000000D3
:1081A000A0042000446202000000000050052000EE
:1081B000446202000000000030052000446202001A
:1081C00000000000400520004462020000000000A2
:1081D00000712200E08288001001200010818800D8
:1081E0008C0B0400000000009E63020000000000F1
:1081F000B407200060042000C662020000000000F6
:10820000F30F20000300620044620200000000003F
:108210004822DE0003006200446202000000000009
:1082200020042000C662020000000000300420008C
:1082300044620200000000000002200044620200CC
:108240000000000010042000446202000000000052
:10825000000220004462020000000000C004200070
:10826000446202000000000000022000446202009C
:1082700000000000900420004462020000000000A2
:1082800000022000446202000000000020042000E0
:10829000446202000000000000022000446202006C
:1082A00000000000200520004462020000000000E1
:1082B00000022000446202000000000010042000C0
:1082C000446202000000000000022000446202003C
:1082D0000000000040052000446202000000000091
:1082E0000002200044620200000000009004200010
:1082F000446202000000000000022000446202000C
:1083000000000000F00420004462020000000000B1
:10831000000220004462020000000000E00420008F
:108320004462020000000000340A200060042000C3
:10833000C662020000000000F30F2000030062008C
:1083400044620200000000004822DE0003006200D8
:10835000446202000000000020042000C662020007
:1083600000000000D0022000446202000000000073
:10837000D00220004462020000000000D002200071
:108380004462020000000000D002200044620200AB
:1083900000000000D0022000446202000000000043
:1083A000D00220004462020000000000D002200041
:1083B0004462020000000000D0022000446202007B
:1083C00000000000D0022000446202000000000013
:1083D000D00220004462020000000000D002200011
:1083E0004462020000000000D0022000446202004B
:1083F00000000000D00220004462020000000000E3
:10840000D00220004462020000000000D0022000E0
:108410004462020000000000D0022000446202001A
:1084200000000000D00220004462020000000000B2
:10843000D00220004462020000000000D0022000B0
:108440004462020000000000D002200044620200EA
:1084500000000000D0022000446202000000000082
:10846000D424200060042000C66202000000000046
:10847000F30F2000030062004462020000000000CD
:108480004822DE0003006200446202000000000097
:1084900020042000C6620200000000003005200019
:1084A0004462020000000000000520004462020057
:1084B00000000000500420004462020000000000A0
:1084C000500420004462020000000000400420002C
:1084D0004462020000000000242720006004200005
:1084E000C662020000000000F30F200003006200DB
:1084F00044620200000000004822DE000300620027
:10850000446202000000000020042000C662020055
:1085100000000000D00620004462020000000000BD
:10852000D00620004462020000000000F00220009B
:1085300044620200000000000007200044620200C4
:10854000000000005007200044620200000000000C
:10855000C006200044620200000000003007200036
:108560004462020000000000500620004462020045
:108570000000000000022000446202000000000031
:10858000E0808000808188005C67020000000000BD
:10859000508280000103200001004000446202007C
:1085A0000000000060828000010320000100400004
:1085B000446202000000000070828000010320007D
:1085C0000100400044620200000000008082800040
:1085D000010320000100400044620200000000008E
:1085E0008448200060042000C662020000000000F1
:1085F000F30F20000300620044620200000000004C
:108600004822DE0003006200446202000000000015
:1086100020042000C662020000000000D0042000F8
:1086200044620200000000001004200044620200C6
:1086300000000000900420004462020000000000DE
:10864000E00420004462020000000000000220005C
:108650004462020000000000D004200044620200D6
:1086600000000000500420004462020000000000EE
:10867000E0042000446202000000000050052000D9
:108680004462020000000000444920006004200011
:10869000C662020000000000F30F20000300620029
:1086A00044620200000000004822DE000300620075
:1086B000446202000000000020042000C6620200A4
:1086C000000000006004200044620200000000007E
:1086D00090042000446202000000000020052000F9
:1086E00044620200000000003005200044620200E5
:1086F000000000004005200044620200000000006D
:10870000000220004462020000000000300520004A
:108710004462020000000000500420004462020095
:1087200000000000C00420004462020000000000BD
:1087300050042000446202000000000030042000C9
:108740004462020000000000400520004462020074
:10875000000000000002200044620200000000004F
:108760009004200044620200000000004005200048
:108770004462020000000000500420004462020035
:1087800000000000D004200044620200000000004D
:1087900000022000446202000000000040052000AA
:1087A0004462020000000000F00420004462020065
:1087B00000000000000220004462020000000000EF
:1087C0001004200044620200000000004004200069
:1087D0004462020000000000A00420004462020085
:1087E000000000005005200044620200000000006C
:1087F0003005200044620200000000004005200017
:10880000446202000000000000712200E082880043
:10881000D0002000108188008C0B040000000000B4
:1088200090C6800031002000010050004220AE00C0
:108830002C44040000000000702102000000000031
:108840001C78020000000000200020001081880039
:10885000444404000000000090C680008100200015
:10886000010050004220AE0044440400000000001B
:10887000702102000000000000022000108188002A
:1088800044440400000000008C0B040000000000C1
:108890008448200060042000C6620200000000003E
:1088A000F30F200003006200446202000000000099
:1088B0004822DE0003006200446202000000000063
:1088C00020042000C6620200000000000002200018
:1088D0004462020000000000000220004462020026
:1088E00000000000000220004462020000000000BE
:1088F000000220004462020000000000000220008C
:1089000044620200000000000002200044620200F5
:10891000000000000002200044620200000000008D
:10892000000220004462020000000000000220005B
:10893000446202000000000044492000600420005E
:10894000C662020000000000F30F20000300620076
:1089500044620200000000004822DE0003006200C2
:10896000446202000000000020042000C6620200F1
:10897000000000000002200044620200000000002D
:1089800000022000446202000000000050052000A8
:108990004462020000000000000520004462020062
:1089A00000000000000220004462020000000000FD
:1089B00000022000446202000000000000022000CB
:1089C0004462020000000000000220004462020035
:1089D00000000000000220004462020000000000CD
:1089E000000220004462020000000000000220009B
:1089F0004462020000000000000220004462020005
:108A0000000000004004200044620200000000005A
:108A1000F004200044620200000000007005200005
:108A20004462020000000000E004200044620200F2
:108A3000000000000002200044620200000000006C
:108A4000000220004462020000000000000220003A
:108A500044620200000000000002200044620200A4
:108A6000000000000002200044620200000000003C
:108A700000022000446202000000000030052000D7
:108A80004462020000000000400520004462020031
:108A900000000000F004200044620200000000001A
:108AA0002005200044620200000000005004200065
:108AB00044620200000000001002200010818800C3
:108AC0008C0B040000000000E08080009082880091
:108AD000B0272000B082880000002000C0828800FB
:108AE000801F02000000000090828000E08088006B
:108AF0008448200060042000C662020000000000DC
:108B0000F30F200003006200446202000000000036
:108B10004822DE0003006200446202000000000000
:108B200020042000C662020000000000D0042000E3
:108B300044620200000000001004200044620200B1
:108B400000000000900420004462020000000000C9
:108B5000E004200044620200000000000002200047
:108B60004462020000000000D004200044620200C1
:108B700000000000500420004462020000000000D9
:108B8000E0042000446202000000000050052000C4
:108B900044620200000000004449200060042000FC
:108BA000C662020000000000F30F20000300620014
:108BB00044620200000000004822DE000300620060
:108BC000446202000000000020042000C66202008F
:108BD0000000000060042000446202000000000069
:108BE00090042000446202000000000020052000E4
:108BF00044620200000000003005200044620200D0
:108C00000000000040052000446202000000000057
:108C10000002200044620200000000003005200035
:108C20004462020000000000500420004462020080
:108C300000000000C00420004462020000000000A8
:108C400050042000446202000000000030042000B4
:108C5000446202000000000040052000446202005F
:108C6000000000000002200044620200000000003A
:108C70009004200044620200000000004005200033
:108C80004462020000000000500420004462020020
:108C900000000000D0042000446202000000000038
:108CA0000002200044620200000000004005200095
:108CB0004462020000000000F00420004462020050
:108CC00000000000000220004462020000000000DA
:108CD0001004200044620200000000004004200054
:108CE0004462020000000000A00420004462020070
:108CF0000000000050052000446202000000000057
:108D00003005200044620200000000004005200001
:108D1000446202000000000000712200E08288002E
:108D2000D0002000108188008C0B0400000000009F
:108D30009E63020000000000E41120006004200097
:108D4000C662020000000000F30F20000300620072
:108D500044620200000000004822DE0003006200BE
:108D6000446202000000000020042000C6620200ED
:108D70000000000000052000446202000000000026
:108D8000000220004462020000000000F004200005
:108D90004462020000000000000220004462020061
:108DA0000000000070052000446202000000000086
:108DB0000002200044620200000000005004200075
:108DC0004462020000000000000220004462020031
:108DD00000000000200520004462020000000000A6
:108DE0000002200044620200000000000002200097
:108DF0004462020000000000000220004462020001
:108E000000000000F00420004462020000000000A6
:108E10000002200044620200000000006004200004
:108E200044620200000000000002200044620200D0
:108E30000000000060042000446202000000000006
:108E40006414200060042000C662020000000000DC
:108E5000F30F2000030062004462020000000000E3
:108E60004822DE00030062004462020000000000AD
:108E700020042000C662020000000000D002200092
:108E80004462020000000000D002200044620200A0
:108E900000000000D0022000446202000000000038
:108EA000D00220004462020000000000D002200036
:108EB0004462020000000000D00220004462020070
:108EC00000000000D0022000446202000000000008
:108ED000D00220004462020000000000D002200006
:108EE0004462020000000000D00220004462020040
:108EF00000000000D00220004462020000000000D8
:108F0000D00220004462020000000000D0022000D5
:108F10004462020000000000D0022000446202000F
:108F200000000000D00220004462020000000000A7
:108F3000D00220004462020000000000D0022000A5
:108F400044620200000000000423200060042000AE
:108F5000C662020000000000F30F20000300620060
:108F600044620200000000004822DE0003006200AC
:108F7000446202000000000020042000C6620200DB
:108F80000000000000052000446202000000000014
:108F9000F004200044620200000000007005200080
:108FA00044620200000000005004200044620200FD
:108FB00000000000200520004462020000000000C4
:108FC000000220004462020000000000F0042000C3
:108FD00044620200000000006004200044620200BD
:108FE0000000000060042000446202000000000055
:108FF0001425200060042000C6620200000000006A
:10900000F30F200003006200446202000000000031
:109010004822DE00030062004462020000000000FB
:1090200020042000C662020000000000300420007E
:1090300044620200000000001004200044620200AC
:1090400000000000E0042000446202000000000074
:1090500030042000446202000000000050042000A0
:109060004462020000000000C004200044620200CC
:10907000000000006425200060042000C662020099
:1090800000000000F30F20000300620044620200B1
:10909000000000004822DE0003006200446202007B
:1090A0000000000080382100E08288002230EC00BF
:1090B0008C0B04000000000090C68000110020000E
:1090C000010050004220AE006E4804000000000085
:1090D00075AEA900A61B04000000000090C6800029
:1090E00081002000010050004220AE0086480400AC
:1090F000000000007021020000000000200020009D
:1091000010818800A61B0400000000005C10E20033
:109110004220AE009648040000000000200020001D
:109120001081880096480400000000008C0B0400A9
:10913000000000009E63020000000000D411200027
:1091400060042000C662020000000000F30F20004F
:109150000300620044620200000000004822DE00BA
:1091600003006200446202000000000020042000AE
:10917000C6620200000000004004200044620200B9
:109180000000000000022000446202000000000015
:1091900010042000446202000000000000022000D1
:1091A000446202000000000040052000446202000A
:1091B00000000000000220004462020000000000E5
:1091C00010042000446202000000000000022000A1
:1091D000446202000000000000022000446202001D
:1091E00000000000000220004462020000000000B5
:1091F000D0042000446202000000000000022000B1
:1092000044620200000000001004200044620200DA
:109210000000000000022000446202000000000084
:10922000E004200044620200000000000002200070
:1092300044620200000000001004200044620200AA
:109240000000000000022000446202000000000054
:1092500070042000446202000000000000022000B0
:10926000446202000000000050042000446202003A
:109270000000000000022000446202000000000024
:10928000D004200044620200000000000002200020
:10929000446202000000000050042000446202000A
:1092A00000000000000220004462020000000000F4
:1092B000E0042000446202000000000000022000E0
:1092C00044620200000000004005200044620200E9
:1092D000000000005414200060042000C662020058
:1092E00000000000F30F200003006200446202004F
:1092F000000000004822DE00030062004462020019
:109300000000000020042000C662020000000000EF
:10931000D00220004462020000000000D0022000C1
:109320004462020000000000D002200044620200FB
:1093300000000000D0022000446202000000000093
:10934000D00220004462020000000000D002200091
:109350004462020000000000D002200044620200CB
:1093600000000000D0022000446202000000000063
:10937000D00220004462020000000000D002200061
:109380004462020000000000D0022000446202009B
:1093900000000000D0022000446202000000000033
:1093A000D00220004462020000000000D002200031
:1093B0004462020000000000D0022000446202006B
:1093C00000000000D0022000446202000000000003
:1093D000D00220004462020000000000D002200001
:1093E0004462020000000000D0022000446202003B
:1093F00000000000D00220004462020000000000D3
:10940000D00220004462020000000000D0022000D0
:109410004462020000000000D0022000446202000A
:1094200000000000D00220004462020000000000A2
:10943000D00220004462020000000000D0022000A0
:109440004462020000000000D002200044620200DA
:1094500000000000D0022000446202000000000072
:10946000D00220004462020000000000042320001B
:1094700060042000C662020000000000F30F20001C
:109480000300620044620200000000004822DE0087
:10949000030062004462020000000000200420007B
:1094A000C662020000000000300420004462020096
:1094B00000000000C0042000446202000000000020
:1094C000500420004462020000000000100420004C
:1094D00044620200000000002005200044620200F7
:1094E000000000003425200060042000C662020055
:1094F00000000000F30F200003006200446202003D
:10950000000000004822DE00030062004462020006
:109510000000000020042000C662020000000000DD
:1095200030052000446202000000000050042000CA
:109530004462020000000000E004200044620200D7
:10954000000000004004200044620200000000000F
:10955000B440200060042000C66202000000000049
:10956000F30F2000030062004462020000000000CC
:109570004822DE0003006200446202000000000096
:1095800020042000C6620200000000004004200009
:109590004462020000000000500520004462020006
:1095A00000000000D004200044620200000000001F
:1095B00000052000446202000000000084482000F2
:1095C00060042000C662020000000000F30F2000CB
:1095D0000300620044620200000000004822DE0036
:1095E000030062004462020000000000200420002A
:1095F000C662020000000000200420004462020055
:10960000000000001004200044620200000000007E
:10961000300420004462020000000000B00420007A
:10962000446202000000000080382100E0828800CF
:109630002230EC008C0B04000000000090C680007B
:1096400031002000010050004220AE00364B0400E3
:109650000000000070210200000000002000200037
:1096600010818800444D04000000000090C6800076
:1096700011002000010050004220AE005A4B0400AF
:10968000000000000000200000948800000020007E
:1096900010948800D0C68000C0C68800000020005A
:1096A000B0C6880080382100E0828800444D040064
:1096B0000000000090C680008100200001005000E2
:1096C0004220AE00444C0400000000007021020063
:1096D00000000000500420006A6D0200000000003D
:1096E000200420006A6D020000000000000320003A
:1096F0006A6D020000000000800320006A6D020015
:1097000000000000C00420006A6D0200000000009C
:10971000F00620006A6D02000000000070062000C4
:109720006A6D020000000000E00320006A6D020084
:1097300000000000E093800020948800F0938000F7
:109740003094880000002000E09388000000200092
:10975000F093880015EEA90015CEA90015AEA8005B
:1097600000000000000000000000000000000000F9
:10977000000000000000000000000000156EA900BD
:1097800000000000000000000000000000000000D9
:10979000000000000000000000000000800E20001B
:1097A0002C60020000000000000020002C6002007D
:1097B00000000000000020002C60020000000000FB
:1097C000000020002C6002000000000000002000CB
:1097D0002C60020000000000000020002C6002004D
:1097E00000000000000020002C60020000000000CB
:1097F000000020002C6002000000000080600200D9
:1098000000000000BC7902000000000010002000F1
:109810007C32B400000020007EB2B400E0938000EF
:10982000F1938000029480001394800000005100A6
:10983000818059004200AF00FE4B04000000000090
:1098400020948000E093880030948000F09388009A
:1098500015EEA90015CEA90015AEA9000000000064
:1098600000000000000000000000000000000000F8
:10987000000000000000000080382100E082880025
:10988000444D04000000000090C6800071002000DC
:10989000010050004220AE00344D040000000000E2
:1098A0007021020000000000500420006A6D0200D8
:1098B00000000000200420006A6D0200000000008B
:1098C000000320006A6D02000000000080032000F9
:1098D0006A6D020000000000400420006A6D020072
:1098E00000000000500720006A6D02000000000028
:1098F000D00620006A6D0200000000000007200072
:109900006A6D020000000000E00320006A6D0200A2
:1099100000000000E093800020948800F093800015
:109920003094880000002000E093880000002000B0
:10993000F093880015EEA90015CEA90015AEA80079
:109940000000000000000000000000000000000017
:10995000000000000000000000000000156EA900DB
:1099600000000000000000000000000000000000F7
:10997000000000000000000000000000800E200039
:109980002C60020000000000000020002C6002009B
:1099900000000000000020002C6002000000000019
:1099A000000020002C6002000000000000002000E9
:1099B0002C60020000000000000020002C6002006B
:1099C00000000000000020002C60020000000000E9
:1099D000000020002C6002000000000080600200F7
:1099E00000000000BC790200000000001000200010
:1099F0007C32B400000020007EB2B400E09380000E
:109A0000F1938000F2FF2F00F300200000005100CE
:109A1000818059004200AF00EE4C040000000000BD
:109A200020948000E093880030948000F0938800B8
:109A300015EEA90015CEA90015AEA9000000000082
:109A40000000000000000000000000000000000016
:109A5000000000000000000080382100E082880043
:109A6000444D0400000000005C10E2004220AE0003
:109A7000444D0400000000002000200010818800F8
:109A8000444D0400000000008C0B040000000000A6
:109A90009E63020000000000844820006004200053
:109AA000C662020000000000F30F20000300620005
:109AB00044620200000000004822DE000300620051
:109AC000446202000000000020042000C662020080
:109AD00000000000D00420004462020000000000EA
:109AE00010042000446202000000000090042000E6
:109AF0004462020000000000E00420004462020012
:109B0000000000000002200044620200000000008B
:109B1000D004200044620200000000005004200035
:109B20004462020000000000E004200044620200E1
:109B30000000000050052000446202000000000008
:109B4000B400200060042000C66202000000000093
:109B5000F30F2000030062004462020000000000D6
:109B60004822DE00030062004462020000000000A0
:109B700020042000C662020000000000B0062000A1
:109B800044620200000000007006200044620200EF
:109B900000000000F002200044620200000000000B
:109BA000800620004462020000000000B43720005C
:109BB00060042000C662020000000000F30F2000D5
:109BC0000300620044620200000000004822DE0040
:109BD0000300620044620200000000002004200034
:109BE000C662020000000000B006200044620200CD
:109BF0000000000070062000446202000000000027
:109C0000F0022000446202000000000080062000F4
:109C100044620200000000003401200060042000C3
:109C2000C662020000000000F30F20000300620083
:109C300044620200000000004822DE0003006200CF
:109C4000446202000000000020042000C6620200FE
:109C500000000000C0062000446202000000000076
:109C6000F0022000446202000000000020072000F3
:109C7000446202000000000034382000600420002C
:109C8000C662020000000000F30F20000300620023
:109C900044620200000000004822DE00030062006F
:109CA000446202000000000020042000C66202009E
:109CB00000000000C0062000446202000000000016
:109CC000F002200044620200000000002007200093
:109CD0004462020000000000A40120006004200093
:109CE000C662020000000000F30F200003006200C3
:109CF00044620200000000004822DE00030062000F
:109D0000446202000000000020042000C66202003D
:109D100000000000D00620004462020000000000A5
:109D2000C00620004462020000000000F002200093
:109D30004462020000000000D006200044620200DD
:109D400000000000A438200060042000C662020069
:109D500000000000F30F20000300620044620200D4
:109D6000000000004822DE0003006200446202009E
:109D70000000000020042000C66202000000000075
:109D8000D00620004462020000000000C00620004F
:109D90004462020000000000F00220004462020061
:109DA00000000000D0062000446202000000000015
:109DB0000405200060042000C662020000000000CC
:109DC000F30F200003006200446202000000000064
:109DD0004822DE000300620044620200000000002E
:109DE00020042000C66202000000000040052000A0
:109DF00044620200000000001006200044620200DD
:109E00000000000020072000446202000000000063
:109E1000700620004462020000000000500620008E
:109E2000446202000000000040072000446202007B
:109E300000000000A00320004462020000000000B7
:109E40001407200060042000C66202000000000029
:109E5000F30F2000030062004462020000000000D3
:109E60004822DE000300620044620200000000009D
:109E700020042000C662020000000000A0032000B1
:109E8000446202000000000040052000446202001D
:109E900000000000100620004462020000000000E4
:109EA000200720004462020000000000700620002D
:109EB00044620200000000005006200044620200DC
:109EC0000000000040072000446202000000000083
:109ED000040A200060042000C662020000000000A6
:109EE000F30F200003006200446202000000000043
:109EF0004822DE000300620044620200000000000D
:109F000020042000C66202000000000000022000C1
:109F100044620200000000002005200044620200AC
:109F200000000000F0062000446202000000000073
:109F300070072000446202000000000000022000C0
:109F4000446202000000000010032000446202008E
:109F500000000000A0032000446202000000000096
:109F6000140C200060042000C66202000000000003
:109F7000F30F2000030062004462020000000000B2
:109F80004822DE000300620044620200000000007C
:109F900020042000C662020000000000A003200090
:109FA000446202000000000020052000446202001C
:109FB00000000000F00620004462020000000000E3
:109FC0007007200044620200000000000002200030
:109FD00044620200000000001003200044620200FE
:109FE00000000000000220004462020000000000A7
:109FF000040F200060042000C66202000000000080
:10A00000F30F200003006200446202000000000021
:10A010004822DE00030062004462020000000000EB
:10A0200020042000C66202000000000000022000A0
:10A03000446202000000000020052000446202008B
:10A0400000000000F0062000446202000000000052
:10A05000700720004462020000000000000220009F
:10A06000446202000000000020032000446202005D
:10A0700000000000A0032000446202000000000075
:10A080001411200060042000C662020000000000DD
:10A09000F30F200003006200446202000000000091
:10A0A0004822DE000300620044620200000000005B
:10A0B00020042000C662020000000000A00320006F
:10A0C00044620200000000002005200044620200FB
:10A0D00000000000F00620004462020000000000C2
:10A0E000700720004462020000000000000220000F
:10A0F00044620200000000002003200044620200CD
:10A100000000000000022000446202000000000085
:10A110000414200060042000C66202000000000059
:10A12000F30F200003006200446202000000000000
:10A130004822DE00030062004462020000000000CA
:10A1400020042000C662020000000000000220007F
:10A15000446202000000000020052000446202006A
:10A1600000000000F0062000446202000000000031
:10A17000700720004462020000000000000220007E
:10A18000446202000000000030032000446202002C
:10A1900000000000A0032000446202000000000054
:10A1A0001416200060042000C662020000000000B7
:10A1B000F30F200003006200446202000000000070
:10A1C0004822DE000300620044620200000000003A
:10A1D00020042000C662020000000000A00320004E
:10A1E00044620200000000002005200044620200DA
:10A1F00000000000F00620004462020000000000A1
:10A2000070072000446202000000000000022000ED
:10A21000446202000000000030032000446202009B
:10A220000000000000022000446202000000000064
:10A230000419200060042000C66202000000000033
:10A24000F30F2000030062004462020000000000DF
:10A250004822DE00030062004462020000000000A9
:10A2600020042000C662020000000000000220005E
:10A270004462020000000000200520004462020049
:10A2800000000000F0062000446202000000000010
:10A29000700720004462020000000000000220005D
:10A2A00044620200000000004003200044620200FB
:10A2B00000000000A0032000446202000000000033
:10A2C000141B200060042000C66202000000000091
:10A2D000F30F20000300620044620200000000004F
:10A2E0004822DE0003006200446202000000000019
:10A2F00020042000C662020000000000A00320002D
:10A3000044620200000000002005200044620200B8
:10A3100000000000F006200044620200000000007F
:10A3200070072000446202000000000000022000CC
:10A33000446202000000000040032000446202006A
:10A340000000000000022000446202000000000043
:10A35000041E200060042000C6620200000000000D
:10A36000F30F2000030062004462020000000000BE
:10A370004822DE0003006200446202000000000088
:10A3800020042000C662020000000000000220003D
:10A390004462020000000000200520004462020028
:10A3A00000000000F00620004462020000000000EF
:10A3B000700720004462020000000000000220003C
:10A3C00044620200000000005003200044620200CA
:10A3D00000000000A0032000446202000000000012
:10A3E0001420200060042000C6620200000000006B
:10A3F000F30F20000300620044620200000000002E
:10A400004822DE00030062004462020000000000F7
:10A4100020042000C662020000000000A00320000B
:10A420004462020000000000200520004462020097
:10A4300000000000F006200044620200000000005E
:10A4400070072000446202000000000000022000AB
:10A450004462020000000000500320004462020039
:10A460000000000000022000446202000000000022
:10A470000423200060042000C662020000000000E7
:10A48000F30F20000300620044620200000000009D
:10A490004822DE0003006200446202000000000067
:10A4A00020042000C662020000000000000220001C
:10A4B0004462020000000000200520004462020007
:10A4C00000000000F00620004462020000000000CE
:10A4D000700720004462020000000000000220001B
:10A4E0004462020000000000600320004462020099
:10A4F00000000000A00320004462020000000000F1
:10A500001425200060042000C66202000000000044
:10A51000F30F20000300620044620200000000000C
:10A520004822DE00030062004462020000000000D6
:10A5300020042000C662020000000000A0032000EA
:10A540004462020000000000200520004462020076
:10A5500000000000F006200044620200000000003D
:10A56000700720004462020000000000000220008A
:10A570004462020000000000600320004462020008
:10A580000000000000022000446202000000000001
:10A590000428200060042000C662020000000000C1
:10A5A000F30F20000300620044620200000000007C
:10A5B0004822DE0003006200446202000000000046
:10A5C00020042000C66202000000000000022000FB
:10A5D00044620200000000002005200044620200E6
:10A5E00000000000F00620004462020000000000AD
:10A5F00070072000446202000000000000022000FA
:10A600004462020000000000700320004462020067
:10A6100000000000A00320004462020000000000CF
:10A62000142A200060042000C6620200000000001E
:10A63000F30F2000030062004462020000000000EB
:10A640004822DE00030062004462020000000000B5
:10A6500020042000C662020000000000A0032000C9
:10A660004462020000000000200520004462020055
:10A6700000000000F006200044620200000000001C
:10A680007007200044620200000000000002200069
:10A6900044620200000000007003200044620200D7
:10A6A00000000000000220004462020000000000E0
:10A6B000042D200060042000C6620200000000009B
:10A6C000F30F20000300620044620200000000005B
:10A6D0004822DE0003006200446202000000000025
:10A6E00020042000C66202000000000000022000DA
:10A6F00044620200000000002005200044620200C5
:10A7000000000000F006200044620200000000008B
:10A7100070072000446202000000000000022000D8
:10A720004462020000000000800320004462020036
:10A7300000000000A00320004462020000000000AE
:10A74000142F200060042000C662020000000000F8
:10A75000F30F2000030062004462020000000000CA
:10A760004822DE0003006200446202000000000094
:10A7700020042000C662020000000000A0032000A8
:10A780004462020000000000200520004462020034
:10A7900000000000F00620004462020000000000FB
:10A7A0007007200044620200000000000002200048
:10A7B00044620200000000008003200044620200A6
:10A7C00000000000000220004462020000000000BF
:10A7D0000432200060042000C66202000000000075
:10A7E000F30F20000300620044620200000000003A
:10A7F0004822DE0003006200446202000000000004
:10A8000020042000C6620200000000004005200075
:10A8100044620200000000001006200044620200B2
:10A820000000000020072000446202000000000039
:10A830007006200044620200000000005006200064
:10A840004462020000000000400720004462020051
:10A8500000000000A003200044620200000000008D
:10A860001434200060042000C662020000000000D2
:10A87000F30F2000030062004462020000000000A9
:10A880004822DE0003006200446202000000000073
:10A8900020042000C662020000000000A003200087
:10A8A00044620200000000004005200044620200F3
:10A8B00000000000100620004462020000000000BA
:10A8C0002007200044620200000000007006200003
:10A8D00044620200000000005006200044620200B2
:10A8E0000000000040072000446202000000000059
:10A8F000B0002000108188008C0B040000000000D4
:10A9000090C6800031002000010050004220AE00BF
:10A91000D855040000000000702102000000000073
:10A92000A629210000002000001B7800004026001E
:10A93000001B7800C62C210000002000001B7800BE
:10A9400000402600001B7800E62F210000002000B8
:10A95000001B780000402600001B78000633210011
:10A9600000002000001B780000402600001B78003B
:10A970002636210000002000001B78000040260041
:10A98000001B78004639210000002000001B7800E1
:10A9900000402600001B7800663C210000002000DB
:10A9A000001B780000402600001B7800863F210035
:10A9B00000002000001B780000402600001B7800EB
:10A9C000A642210000002000001B78000040260065
:10A9D000001B7800C645210000002000001B780005
:10A9E00000402600001B7800E648210000002000FF
:10A9F000001B780000402600001B7800064C210058
:10AA000000002000001B780000402600001B78009A
:10AA1000264F210000002000001B78000040260087
:10AA2000001B78004652210000002000001B780027
:10AA300000402600001B7800665521000000200021
:10AA4000001B780000402600001B7800865821007B
:10AA500000002000001B780000402600001B78004A
:10AA6000A65B210000002000001B780000402600AB
:10AA7000001B7800C65E210000002000001B78004B
:10AA800000402600001B7800E66121000000200045
:10AA9000001B780000402600001B7800066521009E
:10AAA00000002000001B780000402600001B7800FA
:10AAB0002668210000002000001B780000402600CE
:10AAC000001B7800466B210000002000001B78006E
:10AAD00000402600001B7800666E21000000200068
:10AAE000001B780000402600001B780086712100C2
:10AAF00000002000001B780000402600001B7800AA
:10AB0000A674210000002000001B780000402600F1
:10AB1000001B7800C677210000002000001B780091
:10AB200000402600001B7800E67A2100000020008B
:10AB3000001B780000402600001B7800067E2100E4
:10AB400000002000001B780000402600001B780059
:10AB50002681210000002000001B78000040260014
:10AB6000001B78004684210000002000001B7800B4
:10AB700000402600001B78006687210000002000AE
:10AB8000001B780000402600001B7800868A210008
:10AB900000002000001B780000402600001B780009
:10ABA00020002000108188008E5E0400000000005C
:10ABB000030220006832EC00409380000102200074
:10ABC000810050004200AE00F65504000000000075
:10ABD000D4630200000000000064020000000000D6
:10ABE00068B2EF008E5E040000000000862821009D
:10ABF00040938000210320000100B80000034300BF
:10AC00005693880016407800F10020000100600093
:10AC100011002000810050004220AE002C5604009C
:10AC2000000000001660A6000857040000000000A5
:10AC30001650A700E4570400000000001640A000D2
:10AC40001650A600F2570400000000001640A100B4
:10AC5000E4570400000000005693800081002000AB
:10AC60000683400016027800A00020000002420087
:10AC700060042000C662020000000000F30F200004
:10AC80000300620044620200000000004822DE006F
:10AC90000300620044620200000000002004200063
:10ACA000C662020000000000C003200044620200EF
:10ACB0000000000040042000446202000000000088
:10ACC00050042000446202000000000060042000E4
:10ACD0004462020000000000E00320004462020021
:10ACE0000000000056938000810020000683400091
:10ACF00016027800100120000002420060042000CB
:10AD0000C662020000000000F30F20000300620092
:10AD100044620200000000004822DE0003006200DE
:10AD2000446202000000000020042000C66202000D
:10AD30000000000000022000446202000000000049
:10AD4000C003200044620200000000004004200014
:10AD5000446202000000000050042000446202002F
:10AD600000000000600420004462020000000000B7
:10AD7000E0032000446202000000000056938000BF
:10AD80008100200006834000160278009001200018
:10AD90000002420060042000C662020000000000C1
:10ADA000F30F200003006200446202000000000074
:10ADB0004822DE000300620044620200000000003E
:10ADC00020042000C662020000000000C003200032
:10ADD00044620200000000004004200044620200BF
:10ADE0000000000050042000446202000000000047
:10ADF000600420004462020000000000E003200024
:10AE00004462020000000000E4570400000000005B
:10AE100056938000810020000683400016027800CF
:10AE2000A00020000002420060042000C662020070
:10AE300000000000F30F20000300620044620200E3
:10AE4000000000004822DE000300620044620200AD
:10AE50000000000020042000C66202000000000084
:10AE6000C003200044620200000000003004200003
:10AE70004462020000000000F0042000446202006E
:10AE800000000000D0042000446202000000000026
:10AE9000E00320004462020000000000569380009E
:10AEA0008100200006834000160278001001200077
:10AEB0000002420060042000C662020000000000A0
:10AEC000F30F200003006200446202000000000053
:10AED0004822DE000300620044620200000000001D
:10AEE00020042000C66202000000000000022000D2
:10AEF0004462020000000000C0032000446202001F
:10AF00000000000030042000446202000000000045
:10AF1000F00420004462020000000000D004200081
:10AF20004462020000000000E003200044620200CE
:10AF3000000000005693800081002000068340003E
:10AF400016027800900120000002420060042000F8
:10AF5000C662020000000000F30F20000300620040
:10AF600044620200000000004822DE00030062008C
:10AF7000446202000000000020042000C6620200BB
:10AF800000000000C0032000446202000000000036
:10AF9000300420004462020000000000F0042000A1
:10AFA0004462020000000000D0042000446202005D
:10AFB00000000000E00320004462020000000000E6
:10AFC000E4570400000000008301E9000300E000F2
:10AFD0004220AE00DA550400000000008E5E04003E
:10AFE000000000006812E2004220AE00645A040033
:10AFF0000000000050F627008081880090032000A8
:10B000009081880000002000A0818800E0808000FE
:10B01000B08188003830EF003A30EF00B46E0200A3
:10B02000000000005693800051022000068340007B
:10B0300036407800F10F200001006000B640780033
:10B04000C808DD0002F02F0082806000010070005F
:10B05000B081880036407800F10F200001006000C8
:10B06000C08188003A30EF001E6F0200000000002F
:10B070008081800070838800569380004102200008
:10B0800006834000364078000030A7006E30EF00A5
:10B09000803821006E10E2004220AF00A0C6880078
:10B0A00080162000808188000000200090818800A8
:10B0B00000002000A081880000818000B08188000D
:10B0C00000002000C081880000002000D08188009E
:10B0D000B46E020000000000F0808000B0818800A3
:10B0E00000002000C081880000002000D08188007E
:10B0F000B46E020000000000808180001082880091
:10B100009081800020828800A081800030828800A9
:10B1100000A62E0080818800000020009081880019
:10B1200000002000A081880070838000B08188002A
:10B1300000002000C0818800D0818800B46E020029
:10B140000000000080818000E08188009081800004
:10B15000F0818800A0818000008288000083800048
:10B16000B081880000002000C0818800D081880064
:10B17000B46E02000000000010828000B0818800E0
:10B1800020828000C081880020828000C0818800E9
:10B190001E6F02000000000080818000F0828800A5
:10B1A000569380008100200006834000A405200003
:10B1B00060042000C662020000000000F30F2000BF
:10B1C0000300620044620200000000004822DE002A
:10B1D000030062004462020000000000200420001E
:10B1E000C6620200000000000083800080818800A9
:10B1F0005C67020000000000408280000103200024
:10B200000100400044620200000000005082800003
:10B210000103200001004000446202000000000021
:10B2200060828000010320000100400044620200AF
:10B230000000000070828000010320000100400037
:10B2400044620200000000008082800001032000B0
:10B25000010040004462020000000000A43220000F
:10B2600060042000C662020000000000F30F20000E
:10B270000300620044620200000000004822DE0079
:10B28000030062004462020000000000200420006D
:10B29000C6620200000000000083800080818800F8
:10B2A0005C67020000000000408280000103200073
:10B2B0000100400044620200000000005082800053
:10B2C0000103200001004000446202000000000071
:10B2D00060828000010320000100400044620200FF
:10B2E0000000000070828000010320000100400087
:10B2F0004462020000000000808280000103200000
:10B3000001004000446202000000000056938000EB
:10B310008100200006834000940620006004200085
:10B32000C662020000000000F30F2000030062006C
:10B3300044620200000000004822DE0003006200B8
:10B34000446202000000000020042000C6620200E7
:10B350000000000056938000210120000683400079
:10B3600036407800F20F200002006000964078001E
:10B37000C808DD0002F02F0082806000010070002C
:10B38000808188005C67020000000000408280002D
:10B3900001032000010040004462020000000000A0
:10B3A000508280000103200001004000446202003E
:10B3B00000000000608280000103200001004000C6
:10B3C000446202000000000070828000010320003F
:10B3D0000100400044620200000000008082800002
:10B3E0000103200001004000446202000000000050
:10B3F0009433200060042000C662020000000000B8
:10B40000F30F20000300620044620200000000000D
:10B410004822DE00030062004462020000000000D7
:10B4200020042000C6620200000000005693800045
:10B43000210120000683400036407800F20F2000F2
:10B440000200600096407800C808DD0002F02F007E
:10B450008280600001007000808188005C670200CB
:10B460000000000040828000010320000100400035
:10B4700044620200000000005082800001032000AE
:10B480000100400044620200000000006082800071
:10B49000010320000100400044620200000000009F
:10B4A000708280000103200001004000446202001D
:10B4B00000000000808280000103200001004000A5
:10B4C00044620200000000007083800056938000F8
:10B4D00041012000068340000000E0001100200030
:10B4E0004220AF0001002000014B780056938000FD
:10B4F0002001200000034300F0828000F10F2000B3
:10B5000001006000005B7800F08280004800DE00EF
:10B5100001006000005B780056938000200220004C
:10B52000000343001600780080818800000020009E
:10B5300090818800A081880010828000B0818800FE
:10B5400020828000C081880030828000D081880005
:10B55000B46E020000000000E0818000B08188002D
:10B56000F0818000C081880000828000D081880046
:10B570001E6F020000000000569380006000200053
:10B580000003430080818000000B78005693800008
:10B590008081800001838000010150001670A100AD
:10B5A0004200AE001670A0004200AF00DC5A04005A
:10B5B000000000000201EA00928388005693800098
:10B5C000810020000683400016027800A0002000C1
:10B5D0000002420060042000C66202000000000079
:10B5E000F30F20000300620044620200000000002C
:10B5F0004822DE00030062004462020000000000F6
:10B6000020042000C6620200000000005693800063
:10B610001670A600365B0400000000000210AE00A9
:10B62000365B0400000000000002200044620200BB
:10B630000000000000022000446202000000000040
:10B64000000220004462020000000000000220000E
:10B650004462020000000000000220004462020078
:10B6600000000000825B0400000000005693800090
:10B6700060002000000343001600780080818800ED
:10B680005593800000032000008042001000A700B6
:10B69000C26F0200000000005C67020000000000B2
:10B6A000408280000103200001004000446202004B
:10B6B00000000000508280000103200001004000D3
:10B6C000446202000000000060828000010320004C
:10B6D000010040004462020000000000708280000F
:10B6E000010320000100400044620200000000004D
:10B6F00080828000010320000100400044620200BB
:10B7000000000000945C04000000000016007800B7
:10B71000808188000000200090818800A08188003E
:10B7200056938000810020000683400016027800B6
:10B73000100120000002420060042000C6620200E6
:10B7400000000000F30F20000300620044620200CA
:10B75000000000004822DE00030062004462020094
:10B760000000000020042000C6620200000000006B
:10B7700000818000B081880000002000C081880026
:10B78000D0818800B46E020000000000F0808000CC
:10B79000B081880000002000C0818800D08188002E
:10B7A000B46E02000000000000242400B081880074
:10B7B000F0002000C081880000002000D0818800B7
:10B7C0001E6F0200000000005C6702000000000025
:10B7D000408280000103200001004000446202001A
:10B7E00000000000508280000103200001004000A2
:10B7F000446202000000000060828000010320001B
:10B8000001004000446202000000000070828000DD
:10B81000010320000100400044620200000000001B
:10B820008082800001032000010040004462020089
:10B830000000000056938000810020000683400035
:10B8400016027800900120000002420060042000EF
:10B85000C662020000000000F30F20000300620037
:10B8600044620200000000004822DE000300620083
:10B87000446202000000000020042000C6620200B2
:10B880000000000056938000210220000683400043
:10B8900016007800808188005C67020000000000CC
:10B8A0004082800001032000010040004462020049
:10B8B00000000000508280000103200001004000D1
:10B8C000446202000000000060828000010320004A
:10B8D000010040004462020000000000708280000D
:10B8E000010320000100400044620200000000004B
:10B8F00080828000010320000100400044620200B9
:10B90000000000005693800016407800F1002000EF
:10B910000100600011002000010050004220AE0034
:10B92000065D0400000000005693800081002000A6
:10B93000068340005445200060042000C6620200D7
:10B9400000000000F30F20000300620044620200C8
:10B95000000000004822DE00030062004462020092
:10B960000000000020042000C66202000000000069
:10B9700070838000808188005C6702000000000006
:10B980004082800001032000010040004462020068
:10B9900000000000508280000103200001004000F0
:10B9A0004462020000000000E00220004462020045
:10B9B00000000000608280000103200001004000C0
:10B9C0004462020000000000708280000103200039
:10B9D000010040004462020000000000B0062000A8
:10B9E0004462020000000000D00620004462020011
:10B9F00000000000F002200044620200000000008D
:10BA0000800620004462020000000000569380007F
:10BA10001640A100C43E200060042000C66202005F
:10BA200000000000F30F20000300620044620200E7
:10BA3000000000004822DE000300620044620200B1
:10BA40000000000020042000C66202000000000088
:10BA50004005200044620200000000009006200023
:10BA60004462020000000000D00620004462020090
:10BA700000000000500620004462020000000000A8
:10BA8000A003200044620200000000000002200029
:10BA90004462020000000000218080004808DE00AF
:10BAA0004462020000000000208080004462020026
:10BAB00000000000A003200044620200000000001B
:10BAC000318080004808DE0044620200000000006F
:10BAD000308080004462020000000000A0032000CB
:10BAE0004462020000000000418080004808DE003F
:10BAF00044620200000000004080800044620200B6
:10BB0000000000004441200060042000C6620200E2
:10BB100000000000F30F20000300620044620200F6
:10BB2000000000004822DE000300620044620200C0
:10BB30000000000020042000C66202000000000097
:10BB4000C004200044620200000000001006200033
:10BB5000446202000000000040072000446202002E
:10BB600000000000E002200044620200000000002B
:10BB7000A003200044620200000000000002200038
:10BB80004462020000000000518080004808DE008E
:10BB90004462020000000000508080004462020005
:10BBA00000000000F00D20004462020000000000D0
:10BBB000618080004808DE0044620200000000004E
:10BBC000608080004462020000000000200220002B
:10BBD0004462020000000000718080004808DE001E
:10BBE0004462020000000000708080004462020095
:10BBF000000000007002200044620200000000000B
:10BC0000818080004808DE004462020000000000DD
:10BC1000C443200060042000C6620200000000004F
:10BC2000F30F2000030062004462020000000000E5
:10BC30004822DE00030062004462020000000000AF
:10BC400020042000C662020000000000C0042000A2
:10BC50004462020000000000F0062000446202007E
:10BC600000000000E0062000446202000000000026
:10BC7000700620004462020000000000A0032000C3
:10BC800044620200000000009080800044620200D4
:10BC900000000000A18080004808DE00446202002D
:10BCA00000000000A080800044620200000000004C
:10BCB000F00D20004462020000000000B18080000E
:10BCC0004808DE004462020000000000B0808000EE
:10BCD00044620200000000002002200044620200D2
:10BCE00000000000C18080004808DE0044620200BD
:10BCF00000000000C08080004462020000000000DC
:10BD0000700220004462020000000000D180800028
:10BD10004808DE0044620200000000008C0B0400B2
:10BD200000000000154EA800152EA80015AEA800B2
:10BD300015CEA90015EEA8000000000000000000CC
:10BD4000000000000A610200000000000000000086
:10BD50000000000000000000156EA90000000000B7
:10BD600000000000000000000000000000000000D3
:10BD70000000000000000000800E20002C60020087
:10BD800000000000000020002C6002000000000005
:10BD9000000020002C6002000000000000002000D5
:10BDA0002C60020000000000000020002C60020057
:10BDB00000000000000020002C60020000000000D5
:10BDC000000020002C6002000000000000002000A5
:10BDD0002C600200000000000810200009002D0067
:10BDE0008060020000000000800C78008984E80078
:10BDF0000804E9000800E0004220AE00F05E040004
:10BE00000000000000000000000000000000000032
:10BE1000156EA800000000000000000000000000F7
:10BE20000000000000000000000000000000000012
:10BE3000CC61020000000000156EA90000000000A7
:10BE400000000000000000000000000000000000F2
:10BE50000000000000000000100820002C6002001C
:10BE600000000000000020002C6002000000000024
:10BE7000000020002C6002000000000000002000F4
:10BE80002C60020000000000156EA80000000000F9
:10BE900000000000000000000000000000000000A2
:10BEA0000000000000000000CC6102000000000063
:10BEB000CC61020000000000CC6102000000000024
:10BEC000CC61020000000000156EA9000000000017
:10BED0000000000000000000000000000000000062
:10BEE0000000000000000000400820002C6002005C
:10BEF00000000000000020002C6002000000000094
:10BF0000000020002C600200000000000000200063
:10BF10002C600200000000000810200070002000CB
:10BF2000080040002C600200000000000804E90046
:10BF30000800E0004220AE008E5F04000000000018
:10BF4000156EA800000000000000000000000000C6
:10BF500000000000000000000000000000000000E1
:10BF6000CC61020000000000156EA9000000000076
:10BF700000000000000000000000000000000000C1
:10BF80000000000000000000800820002C6002007B
:10BF900000000000000020002C60020000000000F3
:10BFA000000020002C6002000000000000002000C3
:10BFB0002C60020000000000F08080002C60020075
:10BFC00000000000008180002C60020000000000E2
:10BFD000008380002C6002000000000010838000BD
:10BFE0002C60020000000000208380002C60020012
:10BFF00000000000308380002C6002000000000080
:10C00000408380002C60020000000000508380000C
:10C010002C60020000000000608380002C600200A1
:10C0200000000000156EA8000000000000000000E5
:10C030000000000000000000000000000000000000
:10C0400000000000000000000000000000000000F0
:10C050008C0B0400000000008100200000000000A4
:10C0600000000000000000000000000000000000D0
:10C070000000000000000000548EA9000000000035
:10C0800000000000000000000000000000000000B0
:10C0900000000000000000000000D0000080A600AA
:10C0A00035EEA9000080A70035EEA80000000000D2
:10C0B0000000000000000000000000000000000080
:10C0C0000000000000000000548EA80000000000E6
:10C0D0000000000000000000000000000000000060
:10C0E00000000000000000008100E9000100E00005
:10C0F0004220AE002E600400000000000000060098
:10C10000000020008100200000000000000000006E
:10C11000000000000000000000000000000000001F
:10C1200000000000548EA900000000000000000084
:10C1300000000000000000000000000000000000FF
:10C1400000000000000000000000000000000000EF
:10C15000000000000000D00033CEAF000000A000BF
:10C1600033CEAE000000A10000000000000000007F
:10C1700000000000000000000000000000000000BF
:10C1800000000000548EA800000000000000000025
:10C19000000000000000000000000000000000009F
:10C1A000000000008100E9000100E0004220AE0034
:10C1B000846004000000000000000600156EA90065
:10C1C000000000000000000000000000000000006F
:10C1D000000000000000000000000000700D2000C2
:10C1E0002C600200000000008060020000000000DF
:10C1F000156EA80000000000000000000000000014
:10C20000000000000000000000000000000000002E
:10C2100000000600DE600200000000000070A600C2
:10C220000A610400000000000000A7006061040033
:10C2300000000000156EA9000000000000000000D2
:10C2400000000000000000000000000000000000EE
:10C2500000000000D00320002C600200000000005D
:10C26000A00220002C600200000000000008200056
:10C270002C60020000000000600A20002C60020018
:10C2800000000000156EA800000000000000000083
:10C29000000000000000000000000000000000009E
:10C2A00000000000DE600200000000000070A60038
:10C2B0005261040000000000526104000000000010
:10C2C00000000600FFFF3700A2610200000000002E
:10C2D000942EAA00A261020000000000942EAA0081
:10C2E000A261020000000000942EAA00A2610200D8
:10C2F00000000000942EAA00A261020000000000CD
:10C30000942EAA00A261020000000000942EAA0050
:10C31000A261020000000000942EAA00A2610200A7
:10C3200000000000942EAA00A2610200000000009C
:10C33000942EAA00A261020000000000942EAA0020
:10C3400000000600CC61020000000000CC61020089
:10C3500000000000CC61020000000000CC6102007F
:10C3600000000000CC61020000000000CC6102006F
:10C3700000000000CC61020000000000CC6102005F
:10C3800000000000CC61020000000000CC6102004F
:10C390000000000000000600F6610200000000003E
:10C3A000F661020000000000F661020000000000DB
:10C3B000F661020000000000F661020000000000CB
:10C3C000F661020000000000F661020000000000BB
:10C3D000F661020000000000F661020000000000AB
:10C3E000F6610200000000000000060002022000CA
:10C3F000220888000021EF00524420001208880023
:10C400000068A90002022800220888000068AE0027
:10C410000662040000000000000006001E62020028
:10C4200000000000C1022000810068004220AE0030
:10C430000E62040000000000000006002202AE00B0
:10C440001E620400000000002682BF00F10F2000E1
:10C450000100600034A2B7002222AE003462040062
:10C46000000000002222A900000006000040060093
:10C470000000EB00000778000C000900002F780096
:10C480000007EB0000000600F10F200081006000B3
:10C490000500FC0000F02F00842EB600010078009B
:10C4A000842EB70000000000000000000000000023
:10C4B000000000000000000000000000000000007C
:10C4C0000000000000000000348EA9000000000001
:10C4D000000000000000000000000000000000005C
:10C4E000000000000000000000000000000000004C
:10C4F00034AEA900000000000000000000000000B1
:10C50000000000000000000000000000000000002B
:10C51000000000000000000035AEA900000000008F
:10C52000000000000000000000000000000000000B
:10C5300000000000000000000000000000000000FB
:10C5400000000000000000000000000000000000EB
:10C550000000000035AEA800000000000000000050
:10C5600000000000000000000000000000000000CB
:10C5700000000000000000000000000034AEA80031
:10C58000546302000000000000000600F10F2000CC
:10C59000810060000500FC0000F02F00842EB60032
:10C5A00001007800842EB7000000000000000000A9
:10C5B000000000000000000000000000000000007B
:10C5C000000000000000000000000000348EA80001
:10C5D000000000000000000000000000000000005B
:10C5E000000000000000000000000000000000004B
:10C5F0000000000034AEA9000000000000000000B0
:10C60000000000000000000000000000000000002A
:10C61000000000000000000000000000000000001A
:10C62000000000000000000000000000000000000A
:10C630000000000035AEA90000000000000000006E
:10C6400000000000000000000000000000000000EA
:10C6500000000000000000000000000000000000DA
:10C6600000000000000000000000000000000000CA
:10C6700035AEA8000000000000000000000000002F
:10C6800000000000000000000000000000000000AA
:10C69000000000000000000034AEA8005463020057
:10C6A0000000000000000600000000000000000084
:10C6B000000000000000000000000000000000007A
:10C6C000000000000000000000000000000000006A
:10C6D000000000000000000000000000000000005A
:10C6E000000000000000000000000000000000004A
:10C6F000000000000000000000000000000000003A
:10C700000000000000000000000000000000000029
:10C710000000000000000000000000000000000019
:10C720000000000000000000000000000000000009
:10C73000000000000000060000000600A8630200E0
:10C7400000000000D46302000000000000000600AA
:10C7500060042000C662020000000000000020000B
:10C760004462020000000000000020004462020059
:10C770000000000020042000C6620200000000004B
:10C78000084B20000002200044620200000000006C
:10C790000804E9000800E0004220AE00C263040083
:10C7A000000000000000060060042000C6620200D5
:10C7B00000000000000820004462020000000000A9
:10C7C000500220004462020000000000200420000B
:10C7D000C66202000000000008582200000020008D
:10C7E00044620200000000000804E9000800E000C4
:10C7F0004220AE00EE6304000000000000000600CE
:10C80000840220004E660200000000008407200021
:10C810004E66020000000000840C20004E660200FC
:10C8200000000000841120004E660200000000009D
:10C83000841620004E66020000000000841B2000C9
:10C840004E66020000000000842020004E660200B8
:10C8500000000000842520004E6602000000000059
:10C86000842A20004E66020000000000842F200071
:10C870004E66020000000000843420004E66020074
:10C8800000000000843920004E6602000000000015
:10C89000043C20004E660200000000000446200018
:10C8A0004E6602000000000074052000AC65020026
:10C8B00000000000F4052000AC650200000000004C
:10C8C00064062000AC65020000000000E4062000C1
:10C8D000AC65020000000000740A2000AC65020094
:10C8E00000000000F40A2000AC6502000000000017
:10C8F000640B2000AC65020000000000E40B200087
:10C90000AC65020000000000740F2000AC6502005E
:10C9100000000000F40F2000AC65020000000000E1
:10C9200064102000AC65020000000000E41020004C
:10C93000AC6502000000000074142000AC65020029
:10C9400000000000F4142000AC65020000000000AC
:10C9500064152000AC65020000000000E415200012
:10C96000AC6502000000000074192000AC650200F4
:10C9700000000000F4192000AC6502000000000077
:10C98000641A2000AC65020000000000E41A2000D8
:10C99000AC65020000000000741E2000AC650200BF
:10C9A00000000000F41E2000AC6502000000000042
:10C9B000641F2000AC65020000000000E41F20009E
:10C9C000AC6502000000000074232000AC6502008A
:10C9D00000000000F4232000AC650200000000000D
:10C9E00064242000AC65020000000000E424200064
:10C9F000AC6502000000000074282000AC65020055
:10CA000000000000F4282000AC65020000000000D7
:10CA100064292000AC65020000000000E429200029
:10CA2000AC65020000000000742D2000AC6502001F
:10CA300000000000F42D2000AC65020000000000A2
:10CA4000642E2000AC65020000000000E42E2000EF
:10CA5000AC6502000000000074322000AC650200EA
:10CA600000000000F4322000AC650200000000006D
:10CA700064332000AC65020000000000E4332000B5
:10CA8000AC65020000000000B43F20001266020006
:10CA90000000000054422000126602000000000066
:10CAA000D44420001266020000000000E44520008B
:10CAB0005E65020000000000000006006004200027
:10CAC000C662020000000000F30F200003006200B5
:10CAD00044620200000000004822DE000300620001
:10CAE000446202000000000020042000C662020030
:10CAF000000000000002200044620200000000006C
:10CB00000000060060042000C66202000000000071
:10CB1000F30F2000030062004462020000000000E6
:10CB20004822DE00030062004462020000000000B0
:10CB300020042000C6620200000000000002200065
:10CB40004462020000000000000220004462020073
:10CB5000000000000000060060042000C662020021
:10CB600000000000F30F2000030062004462020096
:10CB7000000000004822DE00030062004462020060
:10CB80000000000020042000C66202000000000037
:10CB900000022000446202000000000000022000A9
:10CBA0004462020000000000000220004462020013
:10CBB000000000000000060060042000C6620200C1
:10CBC00000000000F30F2000030062004462020036
:10CBD000000000004822DE00030062004462020000
:10CBE0000000000020042000C662020000000000D7
:10CBF0000002200044620200000000000002200049
:10CC000044620200000000000002200044620200B2
:10CC1000000000000002200044620200000000004A
:10CC20000000060060042000C66202000000000050
:10CC3000F30F2000030062004462020000000000C5
:10CC40004822DE000300620044620200000000008F
:10CC500020042000C6620200000000000002200044
:10CC60004462020000000000000220004462020052
:10CC700000000000000220004462020000000000EA
:10CC800000022000446202000000000000022000B8
:10CC90004462020000000000000006006004200062
:10CCA000C662020000000000F30F200003006200D3
:10CCB00044620200000000004822DE00030062001F
:10CCC000446202000000000020042000C66202004E
:10CCD000000000000002200044620200000000008A
:10CCE0000002200044620200000000000002200058
:10CCF00044620200000000000002200044620200C2
:10CD00000000000000022000446202000000000059
:10CD10000002200044620200000000000002200027
:10CD20004462020000000000000220004462020091
:10CD30000000000000022000446202000000000029
:10CD400000022000446202000000000000022000F7
:10CD50004462020000000000000220004462020061
:10CD600000000000000220004462020000000000F9
:10CD700000022000446202000000000000022000C7
:10CD80004462020000000000000220004462020031
:10CD900000000000000220004462020000000000C9
:10CDA0000002200044620200000000000002200097
:10CDB0004462020000000000000220004462020001
:10CDC0000000000000022000446202000000000099
:10CDD0000002200044620200000000000002200067
:10CDE00044620200000000000002200044620200D1
:10CDF0000000000000022000446202000000000069
:10CE00000002200044620200000000000002200036
:10CE100044620200000000000002200044620200A0
:10CE20000000000000022000446202000000000038
:10CE30000002200044620200000000000002200006
:10CE40004462020000000000000220004462020070
:10CE50000000000000022000446202000000000008
:10CE600000022000446202000000000000022000D6
:10CE70004462020000000000000220004462020040
:10CE800000000000000220004462020000000000D8
:10CE900000022000446202000000000000022000A6
:10CEA0004462020000000000000220004462020010
:10CEB00000000000000006004830EF004A30EF009C
:10CEC0004C30EF004E30EF005030EF00808180009A
:10CED00001712200010150004200AE007A67040097
:10CEE00000000000020078004830EC006A6704008F
:10CEF00000000000813E2000010150004200AE0011
:10CF00008C67040000000000020078004A30EC004A
:10CF10007C67040000000000410620000101500071
:10CF20004200AE009E67040000000000020078008E
:10CF30004C30EC008E67040000000000A1002000CF
:10CF4000010150004200AE00B06704000000000084
:10CF5000020078004E30EC00A067040000000000E2
:10CF60008082880000000600862821002100200021
:10CF700006834000F20F200002016000025B78008F
:10CF8000C800DE00F20F200002816000025B780022
:10CF9000A62B21002100200006834000F20F200074
:10CFA00002016000025B7800C800DE00F20F200082
:10CFB00002816000025B7800C62E21002100200063
:10CFC00006834000F20F200002016000025B78003F
:10CFD000C800DE00F20F200002816000025B7800D2
:10CFE000E63121002100200006834000F20F2000DE
:10CFF00002016000025B7800C800DE00F20F200032
:10D0000002816000025B78000635210021002000CB
:10D0100006834000F20F200002016000025B7800EE
:10D02000C800DE00F20F200002816000025B780081
:10D03000263821002100200006834000F20F200046
:10D0400002016000025B7800C800DE00F20F2000E1
:10D0500002816000025B7800463B21002100200035
:10D0600006834000F20F200002016000025B78009E
:10D07000C800DE00F20F200002816000025B780031
:10D08000663E21002100200006834000F20F2000B0
:10D0900002016000025B7800C800DE00F20F200091
:10D0A00002816000025B780086412100210020009F
:10D0B00006834000F20F200002016000025B78004E
:10D0C000C800DE00F20F200002816000025B7800E1
:10D0D000A64421002100200006834000F20F20001A
:10D0E00002016000025B7800C800DE00F20F200041
:10D0F00002816000025B7800C64721002100200009
:10D1000006834000F20F200002016000025B7800FD
:10D11000C800DE00F20F200002816000025B780090
:10D12000E64A21002100200006834000F20F200083
:10D1300002016000025B7800C800DE00F20F2000F0
:10D1400002816000025B7800064E21002100200071
:10D1500006834000F20F200002016000025B7800AD
:10D16000C800DE00F20F200002816000025B780040
:10D17000265121002100200006834000F20F2000EC
:10D1800002016000025B7800C800DE00F20F2000A0
:10D1900002816000025B78004654210021002000DB
:10D1A00006834000F20F200002016000025B78005D
:10D1B000C800DE00F20F200002816000025B7800F0
:10D1C000665721002100200006834000F20F200056
:10D1D00002016000025B7800C800DE00F20F200050
:10D1E00002816000025B7800865A21002100200045
:10D1F00006834000F20F200002016000025B78000D
:10D20000C800DE00F20F200002816000025B78009F
:10D21000A65D21002100200006834000F20F2000BF
:10D2200002016000025B7800C800DE00F20F2000FF
:10D2300002816000025B7800C660210021002000AE
:10D2400006834000F20F200002016000025B7800BC
:10D25000C800DE00F20F200002816000025B78004F
:10D26000E66321002100200006834000F20F200029
:10D2700002016000025B7800C800DE00F20F2000AF
:10D2800002816000025B7800066721002100200017
:10D2900006834000F20F200002016000025B78006C
:10D2A000C800DE00F20F200002816000025B7800FF
:10D2B000266A21002100200006834000F20F200092
:10D2C00002016000025B7800C800DE00F20F20005F
:10D2D00002816000025B7800466D21002100200081
:10D2E00006834000F20F200002016000025B78001C
:10D2F000C800DE00F20F200002816000025B7800AF
:10D30000667021002100200006834000F20F2000FB
:10D3100002016000025B7800C800DE00F20F20000E
:10D3200002816000025B78008673210021002000EA
:10D3300006834000F20F200002016000025B7800CB
:10D34000C800DE00F20F200002816000025B78005E
:10D35000A67621002100200006834000F20F200065
:10D3600002016000025B7800C800DE00F20F2000BE
:10D3700002816000025B7800C67921002100200054
:10D3800006834000F20F200002016000025B78007B
:10D39000C800DE00F20F200002816000025B78000E
:10D3A000E67C21002100200006834000F20F2000CF
:10D3B00002016000025B7800C800DE00F20F20006E
:10D3C00002816000025B78000680210021002000BD
:10D3D00006834000F20F200002016000025B78002B
:10D3E000C800DE00F20F200002816000025B7800BE
:10D3F000268321002100200006834000F20F200038
:10D4000002016000025B7800C800DE00F20F20001D
:10D4100002816000025B7800468621002100200026
:10D4200006834000F20F200002016000025B7800DA
:10D43000C800DE00F20F200002816000025B78006D
:10D44000668921002100200006834000F20F2000A1
:10D4500002016000025B7800C800DE00F20F2000CD
:10D4600002816000025B7800000006004200F800C4
:10D47000801F7800811F7800821F7800A0838000C1
:10D480000080E800C21321000201500001003A00B0
:10D4900080072100B1838000810050004220AF004E
:10D4A000606A040000000000311180000168A900DA
:10D4B00001087800A0838800646A0400000000006E
:10D4C000311180000168A900208180000000D00097
:10D4D000E20320000200600000060100FA6A040076
:10D4E000000000000A6B040000000000206B040034
:10D4F00000000000366B0400000000004C6B0400CC
:10D5000000000000626B040000000000786B040063
:10D51000000000008E6B040000000000986B040007
:10D5200000000000A46B040000000000AE6B0400CB
:10D5300000000000BA6B040000000000C46B04008F
:10D5400000000000D06B040000000000E46B040049
:10D5500000000000EE6B040000000000FA6B040005
:10D5600000000000046C040000000000106C0400C7
:10D5700000000000166C040000000000206C040095
:10D58000000000002C6C040000000000406C04004F
:10D59000000000004A6C040000000000606C040001
:10D5A000000000006A6C040000000000746C0400BD
:10D5B00000000000806C0400000000008A6C040081
:10D5C00000000000966C0400000000009C6C040049
:10D5D00000000000A66C040000000000B26C040013
:10D5E00000000000C66C040000000000D06C0400C5
:10D5F0000000000042022000028168004220AE00CC
:10D60000066B0400000000002430EC00E66C04000F
:10D610000000000072042000028168004220AE0079
:10D620001A6B0400000000002430EC001C6B0400A6
:10D63000000000002430EF00E66C04000000000051
:10D6400002052000028168004220AE00306B040019
:10D65000000000002430EC00326B040000000000E9
:10D660002430EF00E66C040000000000720420008B
:10D67000028168004220AE00466B040000000000FA
:10D680002430EC00486B0400000000002430EF0060
:10D69000E66C0400000000007204200002816800B3
:10D6A0004220AE005C6B0400000000002430EC005F
:10D6B0005E6B0400000000002430EF00E66C040004
:10D6C0000000000012042000028168004220AE0029
:10D6D000726B0400000000002430EC00746B040046
:10D6E000000000002430EF00E66C040000000000A1
:10D6F000C2022000028168004220AE00886B040054
:10D70000000000002430EC008A6B040000000000E0
:10D710002430EF00E66C040000000000C808DD00C3
:10D72000218088002430EC00E66C0400000000003A
:10D730002080800081007000218088002430EC006F
:10D74000E66C040000000000C808DD00318088009D
:10D750002430EC00E66C0400000000003080800003
:10D7600081007000318088002430EC00E66C0400F9
:10D7700000000000C808DD00418088002430EC0073
:10D78000E66C040000000000408080008100700012
:10D79000418088002430EC00E66C040000000000AA
:10D7A000C2022000028168004220AE00E06B04004B
:10D7B000000000002430EC00E06B040000000000DA
:10D7C000E66C040000000000C808DD0051808800FD
:10D7D0002430EC00E66C0400000000005080800063
:10D7E00081007000518088002430EC00E66C040059
:10D7F00000000000C808DD00618088002430EC00D3
:10D80000E66C040000000000608080008100700071
:10D81000618088002430EC00E66C04000000000009
:10D820002430EC00E66C040000000000C808DD00B5
:10D83000718088002430EC00E66C040000000000D9
:10D840007080800081007000718088002430EC00BE
:10D85000E66C040000000000C202200002816800A3
:10D860004220AE003C6C0400000000002430EC00BC
:10D870003C6C040000000000E66C040000000000A6
:10D88000C808DD00818088002430EC00E66C0400CC
:10D8900000000000C2022000028168004220AE00A9
:10D8A0005A6C0400000000002430EC005C6C0400A2
:10D8B000000000002430EF00E66C040000000000CF
:10D8C000C808DD00918088002430EC00E66C04007C
:10D8D00000000000C808DD00A18088002430EC00B2
:10D8E000E66C040000000000A08080008100700051
:10D8F000A18088002430EC00E66C040000000000E9
:10D90000C808DD00B18088002430EC00E66C04001B
:10D9100000000000B080800081007000B1808800AD
:10D920002430EC00E66C0400000000002430EC0021
:10D93000E66C040000000000C808DD00C18088001B
:10D940002430EC00E66C040000000000C080800081
:10D9500081007000C18088002430EC00E66C040077
:10D9600000000000C2022000028168004220AE00D8
:10D97000C26C0400000000002430EC00C26C040003
:10D9800000000000E66C040000000000C808DD0094
:10D99000D18088002430EC00E66C04000000000018
:10D9A000C2022000028168004220AE00E06C040048
:10D9B000000000002430EF00E26C040000000000D2
:10D9C0002430EF00E66C0400000000004F017800F6
:10D9D000CF0078004F0078004200F90000400600B8
:10D9E0004200F800801F7800811F7800821F7800B5
:10D9F000A86D0200000000004F017800CF00780001
:10DA00004F0078004200F900004006002222A900E1
:10DA10000828A900004006003222A9000848A900F1
:10DA2000004006004200F800801F7800811F780047
:10DA3000821F78000E6E0200000000004F01780087
:10DA4000CF0078004F0078004200F9000040060047
:10DA50004200F800801F7800811F7800821F780044
:10DA6000DA6D0200000000004F017800CF0078005E
:10DA70004F0078004200F900004006005222A90041
:10DA80000A28A90000400600E0898000F08988008B
:10DA9000F1898000010050004220AE00446D040076
:10DAA000000000000000060021908000800878003F
:10DAB0008180E800822621000281500001003A00A6
:10DAC0008120210021908800158EA9002A68A800D5
:10DAD00000000600018D80008100E8003220210056
:10DAE0000281500001003A00411A2100128D80008D
:10DAF000028150004220AF00766D0400000000005B
:10DB000080487800018D880023E8A8000000060006
:10DB1000F1898000E0898000010050004200A900E6
:10DB20004220AF00A66D0400000000008180E800E4
:10DB3000021A21000281500001003A000114210064
:10DB400011007800F18988004200A800000006005A
:10DB5000118D8000008D8000010050004220AF0038
:10DB6000D06D0400000000003322AF00D86D040027
:10DB7000000000001140780034E2B7008100E800A6
:10DB8000322021000281500001003A00411A210098
:10DB9000118D8800956EAA000C6E04000000000034
:10DBA0003302AE00D86D04000000000023E8A90095
:10DBB000000006003190800020908000010050009D
:10DBC0004220AF00026E0400000000005322AF00AC
:10DBD0000C6E04000000000011007800A012880004
:10DBE0008180E800822621000281500001003A0075
:10DBF0008120210031908800958EAA000C6E0400CF
:10DC0000000000005302AE000C6E04000000000093
:10DC10002A68A900158EA800000006002A68AF0037
:10DC2000366E040000000000E08980000080E800FB
:10DC3000021A21000201500001003A0000142100E4
:10DC4000F1898000810050004220AF00366E040050
:10DC500000000000B11280000A48A9000108780005
:10DC6000E08988003A6E040000000000B1128000D4
:10DC70000A48A900000006000000000000000000A3
:10DC800000000000000000003C6E040000000000E6
:10DC90000000000000000000000000000000000084
:10DCA000486E0400000000000000000000000000BA
:10DCB0000000000000000000546E0400000000009E
:10DCC0000000000000000000000000000000000054
:10DCD000606E040000000000000000000000000072
:10DCE00000000000000000006C6E04000000000056
:10DCF0000000000000000000000000000000000024
:10DD0000786E040000000000000000000000000029
:10DD10000000000000000000846E0400000000000D
:10DD200000000000000000000000000000000000F3
:10DD3000906E0400000000000000000000000000E1
:10DD400000000000000000009C6E040000000000C5
:10DD500000000000000000000000000000000000C3
:10DD60000002040000000000801F7800811F78007E
:10DD7000821F7800831F7800841F7800851F780039
:10DD8000861F7800881F7800891F78008A1F780016
:10DD90008181800092818000A3818000B481800015
:10DDA000C5818000D68180000004EB008004EB0078
:10DDB0000005EB00040CB800888188009981880078
:10DDC0003430EF000414B800080078003230B4009A
:10DDD0000900780034B0B400041CB80008007800D2
:10DDE0003430B400050CB800080078003230B400BC
:10DDF0000900780034B0B4000514B80008007800B9
:10DE00003430B400060CB800080078003430B40098
:10DE10004F057800CF0478004F0478004F03780056
:10DE2000CF0278004F027800CF0178004F017800D0
:10DE3000CF0078004F00780000000600801F7800B7
:10DE4000811F7800821F7800841F7800851F78006A
:10DE5000861F7800881F7800891F78008A1F780045
:10DE60000003200070818800808180009181800003
:10DE7000A2818000B4818000C5818000D6818000AD
:10DE80000004EB008004EB000005EB004200A90059
:10DE90002C10AF004200A8000080D2008180D20088
:10DEA0000281D2000884D2008984D2000A85D2007F
:10DEB0000404540085845C0006055D002C10A90054
:10DEC0004200AF002C10A8000300310004044400FD
:10DED00085844C0006054D002E30ED002E10E2002A
:10DEE0004220AE00466F0400000000004200A9007E
:10DEF0002C10AF004200A8000080D2008180D20028
:10DF00000281D2008081880091818800A2818800EE
:10DF10004F057800CF0478004F0478004F03780055
:10DF2000CF0278004F0278004F017800CF007800D0
:10DF30004F0078000000060000000600801F7800F7
:10DF4000B08180003030B400C081800032B0B400B5
:10DF5000D081800034B0B4004F007800000006008B
:10DF6000801F7800B08180003030B500C081800013
:10DF700032B0B500D081800034B0B5004F007800D9
:10DF800000000600000006001000A100B0072000FD
:10DF9000E66F02000000000040938000E66F020080
:10DFA00000000000C0022000E66F02000000000038
:10DFB00016007800E66F020000000000D007200085
:10DFC000E66F02000000000000000600C1C68000ED
:10DFD000800878008180E80042EB21000281500037
:10DFE00001003A00C18D2100C1C68800D6B8EC00FE
:10DFF00000000600D1C68000110078008180E80092
:10E0000042EB21000281500001003A00C18D210045
:10E01000D1C688000000060005EEA800801F780029
:10E02000811F7800821F7800831F7800841F78008A
:10E03000851F7800861F78007030ED007010E200B8
:10E040004220AE005270040000000000803E20001C
:10E05000808388005270040000000000030220004A
:10E0600082282100030078000000E900210320003D
:10E070000100B800000141001260A60048700400D1
:10E080000000000000032000000141001200A00079
:10E090008301E9000300E0004220AE00307004007C
:10E0A0000000000040C680000000D000E101200018
:10E0B00001006000000601009C70040000000000E8
:10E0C000AE70040000000000D270040000000000E8
:10E0D000F670040000000000207104000000000041
:10E0E0009C700400000000009C7004000000000010
:10E0F0009C700400000000009C7004000000000000
:10E100009C700400000000009C70040000000000EF
:10E110009C700400000000009C70040000000000DF
:10E120009C700400000000009C70040000000000CF
:10E130009C70040000000000CA38EF00CCB8EF006B
:10E14000850EA800852EA900854EA900856EA90020
:10E15000C838EC00E27104000000000050C68000E6
:10E16000838EAE0060C688000000E80083AEAE007B
:10E1700060C688000000E80083CEAE0060C688005C
:10E180000000E80050C68800850EA900852EA80072
:10E19000854EA900856EA900C838EC00E271040024
:10E1A0000000000050C68000838EAE0060C688006C
:10E1B0000000E80083AEAE0060C688000000E80002
:10E1C00083CEAE0060C688000000E80050C688001C
:10E1D000850EA900852EA900854EA800856EA90090
:10E1E000C838EC00E27104000000000050C6800056
:10E1F000838EAE0060C688000000E80083AEAE00EB
:10E2000060C688000000E80083CEAE0060C68800CB
:10E210000000E80050C68800850EA900000000003C
:10E22000852EA90000000000854EA9000000000016
:10E23000856EA800C838EC00E27104000000000000
:10E2400050C68000838EAE0060C688000000E800E3
:10E25000C838EF0060C6800081C680000101500010
:10E260004220AF00407104000000000080C688001A
:10E27000A000200070C68800E271040000000000C9
:10E28000CE18E2004220AF00DE7104000000000062
:10E29000CE38ED00CE18E2004220AE00DE71040060
:10E2A000000000004200DD00C1032000010060000A
:10E2B000000601002000200090C68800DE710400E6
:10E2C000000000001000200090C68800DE710400ED
:10E2D000000000000000200090C68800DE710400ED
:10E2E000000000003000200090C68800DE710400AD
:10E2F000000000004000200090C68800DE7104008D
:10E30000000000005000200090C68800DE7104006C
:10E31000000000008000200090C68800DE7104002C
:10E32000000000007000200090C68800DE7104002C
:10E33000000000006000200090C68800DE7104002C
:10E34000000000009000200090C68800DE710400EC
:10E3500000000000000000000000000000000000BD
:10E3600000000000000000000000000000000000AD
:10E37000000000000000000000000000000000009D
:10E38000000000000000000000000000000000008D
:10E39000000000000000000000000000000000007D
:10E3A000000000000000000000000000000000006D
:10E3B00000000000F0FF2F0090C68800E27104000A
:10E3C000000000005C10E2004220AE005C30ED0076
:10E3D00010818000B1002000010050004220AF00F9
:10E3E000FE710400000000000230A9008038210006
:10E3F000A0C688000E72040000000000D438ED00B2
:10E40000D418E2004220AE000E72040000000000AA
:10E4100080382100A0C688000230A80060938000E8
:10E420000000D000E10320000100600000060100B0
:10E43000B072040000000000BC7204000000000084
:10E440001A73040000000000807304000000000044
:10E45000B673040000000000EC730400000000002C
:10E4600042740400000000005C740400000000001E
:10E47000C074040000000000F674040000000000F6
:10E480002E750400000000007075040000000000FC
:10E49000CC75040000000000EA75040000000000D4
:10E4A0003C760400000000007C76040000000000C0
:10E4B000B276040000000000E876040000000000CE
:10E4C0003E77040000000000B0720400000000006D
:10E4D000B072040000000000B072040000000000F0
:10E4E000B072040000000000B072040000000000E0
:10E4F000B072040000000000B072040000000000D0
:10E50000B072040000000000B072040000000000BF
:10E51000B072040000000000B072040000000000AF
:10E52000B072040000000000B0720400000000009F
:10E53000B072040000000000B0720400000000008F
:10E54000B072040000000000B0720400000000007F
:10E55000B072040000000000B0720400000000006F
:10E560006EB2EF007AB2EF001000200060938800D6
:10E570005C77040000000000030220006E32EC0013
:10E580007093800001022000010050004200AE00A4
:10E59000D6720400000000006EB2EF00D000200030
:10E5A0006093880016730400000000008228210098
:10E5B00070938000210320000100B8000001410099
:10E5C0008293880012407800F10020000100600072
:10E5D0004220AF0004730400000000001260A60097
:10E5E00004730400000000001240A700047304003C
:10E5F000000000001250A00020002000609388005E
:10E6000016730400000000008301E9000300E0002D
:10E610004220AE00BE72040000000000D0002000C6
:10E620006093880016730400000000005C7704000B
:10E630000000000086938000446D0200000000008E
:10E64000709380000000E8000110200001007000BD
:10E65000546D0200000000000002EB0056407800FC
:10E660004400DE00F100200001006000800278001C
:10E6700004024000546D0200000000008502E80022
:10E680001000200004024000546D02000000000051
:10E690000000200004024000546D02000000000051
:10E6A000869380002001200000034300364078005C
:10E6B00004024000546D0200000000008502E900E1
:10E6C0000500E0004220AE00567304000000000088
:10E6D0000480EA00F10F200001006000546D020088
:10E6E000000000008693800020032000A093880093
:10E6F00030002000609388005C7704000000000078
:10E70000886D0200000000004200AF00A07304000A
:10E71000000000007412E2004220AF002E740400DA
:10E72000000000007432ED007412E2004220AE00DE
:10E73000B2730400000000002E740400000000000A
:10E7400001102000810068004220AE002E740400F9
:10E75000000000004000200060938800B2730400B5
:10E76000000000003E74040000000000886D0200FC
:10E77000000000004200AF00D6730400000000005B
:10E780007412E2004220AF002E740400000000006A
:10E790007432ED007412E2004220AE00E87304000F
:10E7A000000000002E740400000000001100200092
:10E7B000810068004220AE002E74040000000000BA
:10E7C0005000200060938800E873040000000000FF
:10E7D0003E74040000000000886D0200000000008C
:10E7E0004200AF000C740400000000007412E2004C
:10E7F0004220AF002E740400000000007432ED00CF
:10E800007412E2004220AE001A74040000000000FE
:10E810002E74040000000000E10F20008100680059
:10E820004220AE002E740400000000001E7404009C
:10E83000000000003E740400000000008693800089
:10E840001664A000A0002000A093880060002000B3
:10E85000609388003E7404000000000086938000EE
:10E860001664A100A0002000A0938800C000200032
:10E87000609388003E740400000000005C77040090
:10E88000000000007412E2004220AF005474040043
:10E89000000000007432ED007412E2004220AE006D
:10E8A000587404000000000070002000609388008D
:10E8B0005C7704000000000086938000446D020035
:10E8C00000000000709380000000E80001102000AC
:10E8D00001007000546D0200000000002630EF00BF
:10E8E00056407800F100200001006000B0938800DD
:10E8F000010420000100700031818000810040008F
:10E9000031818800546D0200000000007632EC0076
:10E91000100020003181800081004000318188009A
:10E92000546D0200000000000001200031818000D1
:10E930008100400031818800546D02000000000019
:10E94000308180000080EA00F10F200001006000AB
:10E95000546D020000000000869380002002200019
:10E96000000343009693880020032000A0938800B2
:10E9700080002000609388005C77040000000000A5
:10E98000886D0200000000004200AF00E074040047
:10E99000000000007412E2004220AF00B8750400CD
:10E9A000000000007432ED007412E2004220AE005C
:10E9B000F274040000000000B875040000000000BC
:10E9C00001102000810068004220AE00B8750400EC
:10E9D000000000009000200060938800F2740400A2
:10E9E00000000000C875040000000000886D0200EF
:10E9F000000000004200AF00167504000000000097
:10EA00007412E2004220AF00B8750400000000005C
:10EA10007432ED007412E2004220AE002A75040048
:10EA200000000000B8750400000000001100200084
:10EA3000810068004220AE00B875040000000000AC
:10EA4000C0938800A0002000609388002A7504000D
:10EA500000000000C875040000000000886D02007E
:10EA6000000000004200AF004E75040000000000EE
:10EA70007412E2004220AF00B875040000000000EC
:10EA80007432ED007412E2004220AE006C75040096
:10EA900000000000B875040000000000969380009C
:10EAA000005B780096938800C1938000810040004D
:10EAB000C19388007632ED007612E2004220AE006B
:10EAC0006C75040000000000B00020006093880016
:10EAD0006C75040000000000C87504000000000010
:10EAE000886D0200000000004200AF009075040035
:10EAF000000000007412E2004220AF00B87504006C
:10EB0000000000007432ED007412E2004220AE00FA
:10EB1000A475040000000000B875040000000000A7
:10EB2000C19380008180EA00F20F200082806000A3
:10EB3000810050004220AE00B875040000000000C3
:10EB4000A875040000000000C87504000000000063
:10EB5000869380001664A000A0002000A093880087
:10EB6000C000200060938800C87504000000000009
:10EB7000869380001664A100A0002000A093880066
:10EB8000C000200060938800C875040000000000E9
:10EB90005C770400000000007412E2004220AF0025
:10EBA000DE750400000000007432ED007412E20013
:10EBB0004220AE00E6750400000000008293800051
:10EBC0001250A10010002000609388005C770400C0
:10EBD00000000000030220007A32EC00D093800095
:10EBE00001022000010050004200AF007A32EF0025
:10EBF00082282100D0938000210320000100B8006A
:10EC0000000141008293880012407800F10020004A
:10EC1000010060004220AF002676040000000000E2
:10EC20001260A70026760400000000001240A70032
:10EC300026760400000000001250A000E000200032
:10EC40006093880038760400000000008301E9002A
:10EC50000300E0004220AE00EC750400000000005C
:10EC60001000200060938800387604000000000047
:10EC70005C7704000000000086938000446D020071
:10EC800000000000D09380000000E8000110200088
:10EC900001007000546D0200000000000000200020
:10ECA000546D02000000000010002000040240002B
:10ECB000546D02000000000000002000040240002B
:10ECC000546D02000000000000002000546D02009E
:10ECD00000000000E00F2000546D02000000000062
:10ECE00020032000A0938800F0002000609388009B
:10ECF0005C77040000000000886D02000000000046
:10ED00004200AF009C760400000000007412E20094
:10ED10004220AF002A770400000000007432ED00AA
:10ED20007412E2004220AE00AE7604000000000043
:10ED30002A77040000000000011020008100680014
:10ED40004220AE002A7704000000000000012000ED
:10ED500060938800AE760400000000003A7704005B
:10ED600000000000886D0200000000004200AF00BB
:10ED7000D2760400000000007412E2004220AF00CE
:10ED80002A770400000000007432ED007412E200E3
:10ED90004220AE00E4760400000000002A77040060
:10EDA0000000000011002000810068004220AE0039
:10EDB0002A77040000000000100120006093880002
:10EDC000E4760400000000003A7704000000000030
:10EDD000886D0200000000004200AF0008770400C8
:10EDE000000000007412E2004220AF002A77040005
:10EDF000000000007432ED007412E2004220AE0008
:10EE000016770400000000002A77040000000000CC
:10EE1000E10F2000810068004220AE002A77040044
:10EE2000000000001A770400000000003A77040098
:10EE300000000000869380001664A000A00020005F
:10EE4000A093880020012000609388003A77040096
:10EE500000000000869380001664A100A00020003E
:10EE6000A093880020012000609388003A77040076
:10EE7000000000005C770400000000007412E20053
:10EE80004220AF0050770400000000007432ED0013
:10EE90007412E2004220AE00587704000000000027
:10EEA000829380001250A10010002000609388001F
:10EEB0005C770400000000004F037800CF02780068
:10EEC0004F027800CF0178004F017800CF00780022
:10EED0004F00780005EEA90000E8A90000400600F8
:10EEE000F09380004300DE0000007800156EA9005A
:10EEF0000000000000000000000000000000000012
:10EF000000000000000000000000000010082000C9
:10EF10002C60020000000000F4938000F307200042
:10EF2000030062002C60020000000000E4938000F7
:10EF30004822DE00030062002C6002000000000096
:10EF4000E4938000F30F2000030062002C600200B5
:10EF500000000000156EA800000000000000000086
:10EF600000000000000000000000000000000000A1
:10EF700000000000CC61020000000000CC61020033
:10EF800000000000CC61020000000000CC61020023
:10EF90000000000000000600F09380004300DE0047
:10EFA00000007800156EA9000000000000000000BD
:10EFB0000000000000000000000000000000000051
:10EFC00000000000800820002C600200000000000B
:10EFD000F4938000F3072000030062002C6002001D
:10EFE00000000000E49380004822DE00030062007D
:10EFF0002C60020000000000E4938000F30F20006A
:10F00000030062002C60020000000000156EA800E2
:10F0100000000000000000000000000000000000F0
:10F02000000000000000000000000000CC610200B1
:10F030000000000000000600CC610200000000009B
:10F04000156EA90000000000000000000000000094
:10F0500000000000000000000000000000000000B0
:10F06000100820002C6002000000000000002000BA
:10F070002C60020000000000000020002C60020054
:10F0800000000000000020002C60020000000000D2
:10F09000156EA80000000000000000000000000045
:10F0A0000000000000000000000000000000000060
:10F0B000CC61020000000000CC61020000000000F2
:10F0C000CC61020000000000CC61020000000000E2
:10F0D000156EA90000000000000000000000000004
:10F0E0000000000000000000000000000000000020
:10F0F000400820002C6002000000000000002000FA
:10F100002C60020000000000000020002C600200C3
:10F1100000000000000020002C6002000000000041
:10F12000F4808000F30F2000030062002C600200D6
:10F13000000000004822DE00030062002C60020094
:10F140000000000004818000F30F20000300620033
:10F150002C600200000000004822DE000300620074
:10F160002C6002000000000004838000F30F2000E8
:10F17000030062002C600200000000004822DE0054
:10F18000030062002C600200000000001483800075
:10F19000F30F2000030062002C600200000000005A
:10F1A0004822DE00030062002C6002000000000024
:10F1B00024838000F30F2000030062002C60020013
:10F1C000000000004822DE00030062002C60020004
:10F1D0000000000034838000F30F20000300620071
:10F1E0002C600200000000004822DE0003006200E4
:10F1F0002C6002000000000044838000F30F200018
:10F20000030062002C600200000000004822DE00C3
:10F21000030062002C6002000000000054838000A4
:10F22000F30F2000030062002C60020000000000C9
:10F230004822DE00030062002C6002000000000093
:10F2400064838000F30F2000030062002C60020042
:10F25000000000004822DE00030062002C60020073
:10F2600000000000E4808000F30F20000300620033
:10F270002C600200000000004822DE000300620053
:10F280002C60020000000000E4938000F30F2000D7
:10F29000030062002C600200000000004822DE0033
:10F2A000030062002C60020000000000F493800064
:10F2B000F30F2000030062002C6002000000000039
:10F2C0004822DE00030062002C6002000000000003
:10F2D000000000000000000000000000156EA80003
:10F2E000000000000000000000000000000000001E
:10F2F000000000000000000000000000CC610200DF
:10F3000000000000156EA9000000000000000000D1
:10F3100000000000000000000000000000000000ED
:10F3200000000000800820002C60020000000000A7
:10F33000000020002C6002000000000000002000FF
:10F340002C60020000000000000020002C60020081
:10F3500000000000156EA800000000000000000082
:10F36000000000000000000000000000000000009D
:10F370000000000000000600801F78004400DE004E
:10F38000F100200001006000DC79020000000000B4
:10F390006A6D0200000000004F007800F1002000BC
:10F3A00001006000DC790200000000006A6D0200CC
:10F3B0000000000000000600A100200081005000B5
:10F3C000010320004200AF00710320000100400053
:10F3D000000006000200000003000000050000001D
:10F3E0000A000000001000007C0F000080000000F8
:10F3F00000000000FFFFFF00FFFFFF00FFFFFF0016
:10F40000FFFFFF00FFFFFF00FFFFFF00FFFFFF0008
:10F41000FFFFFF00FFFFFF00FFFFFF00FFFFFF00F8
:10F42000FFFFFF00FFFFFF00FFFFFF00FFFFFF00E8
:10F43000FFFFFF00FFFFFF00FFFFFF00FFFFFF00D8
:0200000400FFFB
:0200000401F009
:100008000300000083000000250000007F000000BE
:0C00180037000000D500000003000000CD
:04002400FF000000D9
:00000001FF
